:100000000C94BB010C945B320C9488320C94E30189
:100010000C94E3010C94E3010C94E3010C94E301D0
:100020000C94E3010C94E3010C94E3010C94CE06D0
:100030000C94E3010C94E3010C94E3010C94E301B0
:100040000C9467310C94E3010C9444060C948006E4
:100050000C94E3010C94E3010C94E3010C94E30190
:100060000C94E3010C94E301084AD73B3BCE016EAC
:1000700084BCBFFDC12F3D6C74319ABD56833DDAFF
:100080003D00C77F11BED9E4BB4C3E916BAAAABE0E
:10009000000000803F05A84CCDB2D44EB93836A937
:1000A000020C50B9918688083CA6AAAA2ABE000074
:1000B00000803F0664EC1B3C04BC163E3BE5B93CAB
:1000C000C93C37C29E5A3D660498083EEA69AAAA0E
:1000D0003E000000803F2020BF0020BF00BF007C0A
:1000E0002020202020202020202020202020202010
:1000F00020202000C8202020202020202020202078
:1001000020C900C8202020202020202020202020BE
:10011000C97C00D820202020202020202020202042
:10012000D97C00C820202020202020202020202032
:10013000C97C00C820202020202020202020202032
:10014000C97C00207265766F00206172737369004C
:100150006D696E6F706F7364206C6962726570692F
:100160006C6F74002020202020BABBBCBDBE7C2058
:1001700020202020CACBCCCDCE7C00626F6F74696A
:100180006E672075703AEDF2F2F2F2F2F2F2F300DD
:1001900062617474657279207761726E696E67202E
:1001A0000074787069642076616C756573006261B3
:1001B000726F2074656D700074656D706469737022
:1001C00020006163746976652000706173736976DD
:1001D000650075617674616C6B2000736574757071
:1001E0002073637265656E7C7C7C0043686172205D
:1001F000446F6E650A00526561647920666F7220F3
:10020000466F6E740A0055706461746520436861BE
:10021000725365740000407A10F35A00A0724E18B1
:10022000090010A5D4E80000E87648170000E40BA8
:1002300054020000CA9A3B000000E1F5050000806E
:10024000969800000040420F000000A086010000C8
:1002500000102700000000E8030000000064000018
:100260000000000A00000000000100000000002C57
:1002700076D888DC674F0823DFC1DFAE59E1B1B71C
:1002800096E5E3E453C63AE651997696E8E6C284E9
:1002900026EB898C9B62ED407C6FFCEFBC9C9F4001
:1002A000F2BAA56FA5F490055A2AF75C936B6CF926
:1002B000676DC11BFCE0E40D47FEF520E6B500D0FC
:1002C000ED902E0300943577050080841E08000011
:1002D000204E0A000000C80C333333330F986E12DF
:1002E000831141EF8D2114893BE65516CFFEE6DBE5
:1002F00018D1844B381BF77C1D901DA4BBE424202F
:100300003284725E228100C9F124ECA1E53D276EA2
:10031000616E00696E660000000000240027002A5C
:100320000000000000250028002B00000000002332
:100330000026002900040404040404040402020248
:100340000202020303030303030102040810204016
:10035000800102040810200102040810200000009F
:100360000700020100000304060000000000000076
:1003700000004F04150811241FBECFEFD8E0DEBFE8
:10038000CDBF14E0A0E0B1E0E8EAFFE602C00590CE
:100390000D92A030B107D9F716E0A0E0B4E001C09B
:1003A0001D92A33BB107E1F713E0C6E7D3E004C019
:1003B0002297FE010E94CE37C237D107C9F70E94AB
:1003C00097330C94D2370C940000FA01AA272830F6
:1003D00051F1203181F1E8946F936E7F6E5F7F4F12
:1003E0008F4F9F4FAF4FB1E03ED0B4E03CD0670F8E
:1003F000781F891F9A1FA11D680F791F8A1F911DE1
:10040000A11D6A0F711D811D911DA11D20D009F430
:1004100068943F912AE0269F11243019305D319372
:10042000DEF6CF010895462F4770405D4193B3E05B
:100430000FD0C9F7F6CF462F4F70405D4A3318F002
:10044000495D31FD4052419302D0A9F7EACFB4E0B3
:10045000A6959795879577956795BA95C9F700976B
:100460006105710508959B01AC010A2E069457950C
:10047000479537952795BA95C9F7620F731F841F63
:10048000951FA01D0895283008F027E03327DA01D2
:10049000990F311D87FD916000966105710539F452
:1004A00032602E5F3D9330E32A95E1F708959F3F38
:1004B00030F080387105610509F03C5F3C5F3D9389
:1004C000913008F08068911DDF93CF931F930F93B5
:1004D000FF92EF92192F987F9695E92F9695969512
:1004E000E90FFF27E159FD4F99273327EE24FF2419
:1004F000A701E70105900894079428F4360FE71E3A
:10050000F81E491F511D660F771F881F991F0694FB
:10051000A1F70590079428F4E70EF81E491F561F0F
:10052000C11D770F881F991F661F0694A1F70590BC
:10053000079428F4F80E491F561FC71FD11D880FB6
:10054000991F661F771F0694A1F70590079420F462
:10055000490F561FC71FD81F990F661F771F881F87
:100560000694A9F784911095177041F0D695C79518
:1005700057954795F794E7941A95C1F7E5E1F2E0AE
:1005800068941590159135916591959105907FE24C
:100590007395E118F10A430B560BC90BD009C0F74C
:1005A000E10CF11E431F561FC91FD01D7EF470338E
:1005B00011F48A95E6CFE894015030F0080F0AF460
:1005C0000027021708F4202F2395022F7A3328F0F2
:1005D00079E37D932A95E9F710C07D932A9589F6F2
:1005E000069497956795379517951794E118F10A32
:1005F000430B560BC90BD00998F023957E91739548
:100600007A3308F070E37C932013B8F77E91706121
:100610007D9330F0839571E37D9370E32A95E1F744
:100620001124EF90FF900F911F91CF91DF919927A7
:1006300087FD90950895CF93DF93BC01823091059B
:1006400010F462E070E0A091B106B091B206ED0145
:1006500040E050E0E0E0F0E021C088819981861719
:10066000970769F48A819B81309719F0938382837D
:1006700004C09093B2068093B106FE0134C068179F
:10068000790738F44115510519F08417950708F4D6
:10069000AC01FE018A819B819C01E9012097E9F66A
:1006A00041155105A9F1CA01861B970B049708F45F
:1006B000BA01E0E0F0E02AC08D919C911197841777
:1006C0009507F9F46417750781F412968D919C9142
:1006D0001397309719F09383828304C09093B206E6
:1006E0008093B106FD0132964CC0CA01861B970B60
:1006F000FD01E80FF91F6193719302978D939C930D
:1007000040C0FD01828193819C01D9011097A1F61F
:100710008091AF069091B006892B41F48091A002A0
:100720009091A1029093B0068093AF064091A202EF
:100730005091A3024115510541F44DB75EB7809128
:100740009E0290919F02481B590B2091AF06309159
:10075000B006CA01821B930B8617970780F0AB0186
:100760004E5F5F4F8417950750F0420F531F509311
:10077000B0064093AF06F9016193719302C0E0E0C7
:10078000F0E0CF01DF91CF910895CF93DF930097F1
:1007900009F450C0EC0122971B821A82A091B10685
:1007A000B091B206109709F140E050E0AC17BD07D8
:1007B00008F1BB83AA83FE0121913191E20FF31F5F
:1007C000AE17BF0779F48D919C911197280F391FAF
:1007D0002E5F3F4F3983288312968D919C911397FA
:1007E0009B838A834115510571F4D093B206C0935F
:1007F000B10620C012968D919C911397AD01009780
:1008000011F0DC01D3CFFA01D383C283219131915E
:10081000E20FF31FCE17DF0769F488819981280F53
:10082000391F2E5F3F4FFA01318320838A819B81DC
:1008300093838283DF91CF910895FC0105906150ED
:1008400070400110D8F7809590958E0F9F1F0895E6
:10085000FC016150704001900110D8F7809590958F
:100860008E0F9F1F08956EBD0DB407FEFDCF8EB590
:1008700008958DE061E00E94B5328BE061E00E9456
:10088000B5328CE060E00E94B5328AE061E00E94FF
:10089000B5321CBC80E58CBD8DB58EB5089580E069
:1008A00094E00E9439040895FC011382128288EEBC
:1008B00093E0A0E0B0E084839583A683B78385EBC3
:1008C00092E0918380830895FC018089803419F43B
:1008D00021E030E002C020E030E0C9010895FC01D1
:1008E000818990E00895FC01648745876687478782
:1008F000089580E090E0089580E090E0089580E021
:1009000090E008950895EF92FF921F93CF93DF93A5
:10091000162F7A0186E060E00E94F43280E094E0D5
:1009200060E00E94330480E094E060E00E943304C1
:1009300080E094E069E00E94330480E094E0612F5D
:100940000E943304C0E0D0E0F701EC0FFD1F1081DE
:1009500080E094E06AE00E94330480E094E06C2F31
:100960000E94330480E094E06BE00E94330480E056
:1009700094E0612F0E9433042196C633D10521F7FC
:1009800080E094E068E00E94330480E094E060EA54
:100990000E94330480E094E060EA0E94330485FD05
:1009A000F9CF80E094E060E00E94330480E094E0BE
:1009B0006CE00E94330486E061E00E94F432DF9133
:1009C000CF911F91FF90EF9008951F93CF93DF93E6
:1009D000EC01162F86E060E00E94F43280E094E0A3
:1009E00060E00E943304112319F0113059F404C05F
:1009F00080E094E0688904C068896C6180E094E0DC
:100A00000E94330486E061E00E94F432DF91CF91CE
:100A10001F910895EF92FF920F931F938EE1489FCD
:100A200070011124E60EF11C86E060E00E94F432B1
:100A300000E014E0C80165E00E943304C8016F2D96
:100A40000E943304C80166E00E943304C8016E2D81
:100A50000E9433041F910F91FF90EF900895EF9241
:100A6000FF920F931F937C0100E014E0C80167E040
:100A70000E943304C8016FEF0E94330486E061E0F6
:100A80000E94F432F70187858F5F87871F910F914E
:100A9000FF90EF900895EF92FF920F931F93FC0148
:100AA000E7848EE1E89E700111248685E80EF11C32
:100AB00086E060E00E94F43200E014E0C80164E0E7
:100AC0000E943304C80163E00E943304C80165E05A
:100AD0000E943304C8016F2D0E943304C80166E0F0
:100AE0000E943304C8016E2D0E9433041F910F91A0
:100AF000FF90EF9008951F93CF93DF93EC01162F93
:100B00006C3731F40E942F05CE010E944B050AC0BC
:100B100080E094E067E00E94330480E094E0612F7D
:100B20000E94330481E090E0DF91CF911F910895FE
:100B30000F931F9386E060E00E94F43200E014E01F
:100B4000C80164E00E943304C80164E00E943304D9
:100B500086E061E00E94F4321F910F9108951F9387
:100B6000CF93DF93EC01188A16E0198B8FE996E09A
:100B700060E973E00E94C730813049F480E4888BDB
:100B800088E0898B86E060E00E94F43202C0188A17
:100B9000198B86E060E00E94F432DF91CF911F91C3
:100BA00008950F931F93CF93DF93EC0186E061E0EC
:100BB0000E94B53282E060E00E94B53282E061E0DE
:100BC0000E94F432CE010E94AF0586E060E00E94F0
:100BD000F43280E094E06CEE0E94330480E094E014
:100BE0006FEF0E943304182F80E094E060E00E94D1
:100BF00033046889626080E094E00E94330462E319
:100C000070E080E090E00E94BD3180E094E06CE60E
:100C10000E9433041F7E80E094E0612F0E94330421
:100C20008889803419F00DE010E002C000E110E086
:100C3000109202041092010417C060910104709197
:100C40000204605F80E094E00E94330480E094E05E
:100C500069E00E943304809101049091020401969E
:100C60009093020480930104809101049091020406
:100C70008017910714F3CE0161E00E94E504DF9133
:100C8000CF911F910F9108951F920F920FB60F925F
:100C900011242F933F934F938F939F93EF93FF9341
:100CA0004091C60020918E0630918F062F5F3F4FF6
:100CB0008091920690919306282339238091900683
:100CC000909191062817390779F080918E069091BE
:100CD0008F06E0919406F0919506E80FF91F408386
:100CE00030938F0620938E06FF91EF919F918F9105
:100CF0004F913F912F910F900FBE0F901F9018951D
:100D00001F920F920FB60F9211242F933F938F9340
:100D10009F93EF93FF9320919806309199068091CD
:100D200096069091970628173907E9F08091980662
:100D300090919906E0919C06F0919D06E80FF91FAD
:100D400080818093C60080919806909199060196C3
:100D500020919A0630919B068223932390939906C3
:100D60008093980610C02091960630919706809146
:100D70009806909199062817390729F48091C100A7
:100D80008F7D8093C100FF91EF919F918F913F9153
:100D90002F910F900FBE0F901F9018951F920F92DA
:100DA0000FB60F9211248F939F938091C30490915B
:100DB000C404892B51F08091C5049091C60401961A
:100DC0009093C6048093C50409C08091C704909194
:100DD000C80401969093C8048093C7049F918F9193
:100DE0000F900FBE0F901F901895CF93DF93482F51
:100DF000EB0180912406833009F45DC0843028F42F
:100E00008130C1F0823058F50AC0853009F4D2C073
:100E1000853008F4A8C0863009F0F2C0E9C04C3330
:100E200009F0EEC081E080932406488384EB809330
:100E30002306E6C0842F90E0E0912306F0E0E82747
:100E4000F927ED53FD4F208120932306887F907072
:100E5000809741F582E080932406498329C0242F9E
:100E600030E0E0912306F0E0E227F327ED53FD4F59
:100E7000808180932306809122068F5F80932206D3
:100E8000823018F43B832A83BBC0922F88272A81A3
:100E90003B81820F931F9B838A830A978F3F910523
:100EA00021F018F010922406ABC083E08093240652
:100EB00010922206A5C0E42FF0E08091230690E076
:100EC000E827F927ED53FD4F808180932306609139
:100ED00022066F5F60932206623089F0633020F44F
:100EE000613009F08DC006C0633091F0643009F0C4
:100EF00087C022C0842F90E0A0E0B0E018C0242F6B
:100F000030E040E050E0542F432F322F222707C01B
:100F1000242F30E040E050E0A901332722278C81C4
:100F20009D81AE81BF81820F931FA41FB51F8C834B
:100F30009D83AE83BF8364C0242F30E040E050E047
:100F4000522F4427332722278C819D81AE81BF8178
:100F5000820F931FA41FB51F8C839D83AE83BF8315
:100F600060932406A5CF242F30E0E0912306F0E023
:100F7000E227F327ED53FD4F808180932306809174
:100F800022068F5F80932206813019F08230C1F5EE
:100F900003C03987288734C0922F88272885398550
:100FA000280F391F398728878A819B810A97F1F09A
:100FB00085E07CCFE42FF0E08091230690E0E827E5
:100FC000F927ED53FD4F808180932306209122065F
:100FD0002F5F2093220630E0FB01E20FF31F4187D1
:100FE0008A819B810A972817390750F086E05ECFE7
:100FF000C75FDE4F4883C950D14087E08093240605
:1010000080912406873069F410922406C75FDE4F72
:10101000909123068881C950D140981711F48A8194
:1010200001C080E0DF91CF9108958F92AF92CF926F
:10103000EF92FF920F931F9389E894E060E045ECF4
:1010400050E024EC30E000EC10E0B1ECEB2EF12CA1
:10105000CC24C394A8E9AA2EF0E28F2E0E94372A4E
:1010600086EA94E00E9454041092B9041092BA04E3
:101070001092BB041092BC041092BD041092BE04E6
:101080001092BF041092C0041092C2041092C104C6
:101090001092B8041F910F91FF90EF90CF90AF90F6
:1010A0008F900895AF92BF92CF92DF92EF92FF920E
:1010B0000F931F93E0908A06F0908B0600918C06A8
:1010C00010918D068FE590E0A0E0B0E0E80EF91EEB
:1010D0000A1F1B1F0E94AF316E157F058007910705
:1010E00008F44EC0A090EE04B090EF04C090F0045D
:1010F000D090F104C601B50120E030E040E85FE3A4
:101100000E943736181694F5E0904206F090430698
:1011100000914406109145060E94AF3120918A0645
:1011200030918B0640918C0650918D06621B730B9B
:10113000840B950B0E940D359B01AC01C601B501D6
:101140000E94423620E030E04AE754E40E947434C2
:101150009B01AC01C801B7010E94A733609342060E
:101160007093430680934406909345060E94AF31E6
:1011700060938A0670938B0680938C0690938D06FD
:101180001F910F91FF90EF90DF90CF90BF90AF90A5
:101190000895DF93CF9300D000D0CDB7DEB7FB0129
:1011A000E80FF91F628583859485258569838A8385
:1011B0009B832C83492F5C81782FCA010F900F905D
:1011C0000F900F90CF91DF910895AF92BF92DF9271
:1011D000EF92FF920F931F93CF93DF938C01809137
:1011E000250680FDE4C0F801F08089E894E06F2DC9
:1011F0000E94182BE801C75FDE4FEF2DF0E0ED53A2
:10120000FD4F80818883F801F18089E894E06F2D9B
:101210000E94182BEF2DF0E0888190E0E827F92755
:10122000ED53FD4F80818883F801F28089E894E0D6
:101230006F2D0E94182BEF2DF0E0888190E0E827B9
:10124000F927ED53FD4F80818883F801F38089E809
:1012500094E06F2D0E94182BEF2DF0E0888190E034
:10126000E827F927ED53FD4F80818883F801F4804A
:1012700089E894E06F2D0E94182BEF2DF0E0888113
:1012800090E0E827F927ED53FD4F80818883F8012E
:101290002481358146815781232F342F452F5527AF
:1012A000F22E89E894E0622F0E94182BEF2DF0E0D7
:1012B000888190E0E827F927ED53FD4F80818883EE
:1012C000F80124813581468157819A0144275527A9
:1012D000F22E89E894E0622F0E94182BEF2DF0E0A7
:1012E000888190E0E827F927ED53FD4F80818883BE
:1012F000F8012481358146815781252F33274427E2
:101300005527F22E89E894E0622F0E94182BEF2DCA
:10131000F0E0888190E0E827F927ED53FD4F8081C8
:10132000888389E894E060E00E94182BE881F0E06F
:10133000ED53FD4F8081888389E894E060E00E944E
:10134000182BE881F0E0ED53FD4F80818883F80190
:10135000828193810B9718F18AE0A82EB12CA00E00
:10136000B11E750112C0F701D1907F0189E894E0A8
:101370006D2D0E94182BED2DF0E0888190E0E8277C
:10138000F927ED53FD4F808188832E2D2A1930E0F7
:10139000F801828193810A972817390720F3075FA4
:1013A0001E4F89E894E0F80160810E94182BDF91BC
:1013B000CF911F910F91FF90EF90DF90BF90AF9072
:1013C0000895DF93CF93CDB7DEB7CA50D1400FB6A3
:1013D000F894DEBF0FBECDBF2CE329836A832AE0D9
:1013E00030E03C832B83FC0184819581A681B78109
:1013F0008D839E83AF83B887CE0101960E94E50856
:10140000C65FDE4F0FB6F894DEBF0FBECDBFCF91E3
:10141000DF9108958FE996E06AE773E00E94C73094
:10142000882331F586E696E6A6E6B0E480932706A3
:1014300090932806A0932906B0932A0680E090E0B6
:10144000A0E8BFE380932B0690932C06A0932D0673
:10145000B0932E0688EE93E09093300680932F068B
:1014600081E8809331068DE8809332068DEF25C0A8
:1014700082E598EBAEE0B0E48093270690932806CF
:10148000A0932906B0932A0685E89BEEA1E5B0E477
:1014900080932B0690932C06A0932D06B0932E06D6
:1014A00080EA94E19093300680932F068BEF80932F
:1014B000310686E6809332068AEF809333060895DC
:1014C000FF920F931F930FE916E0C8016CE773E0DA
:1014D0000E94C73080936E06C8016EE773E00E94D9
:1014E000C73080936F06C80160E873E00E94C73080
:1014F00080934E06C8016EE873E00E94C730809367
:101500006606C8016AE873E00E94C73080936406EB
:10151000C80164E873E00E94C73080937006C80178
:1015200066E873E00E94C73080937106C8016CE8DA
:1015300073E00E94C73080935606C80162E973E0E9
:101540000E94C73080937206C80164E973E00E946C
:10155000C73080935506C80164EF73E00E94C7301E
:10156000F82EC80165EF73E00E94C730382F20E0E5
:101570002F0D311D3093740620937306C80166EF5A
:1015800073E00E94C730F82EC80167EF73E00E9435
:10159000C730382F20E02F0D311D30937606209371
:1015A0007506C80168EF73E00E94C730F82EC801C5
:1015B00069EF73E00E94C730382F20E02F0D311DF6
:1015C0003093780620937706C8016BEF73E00E9492
:1015D000C73080934D061F910F91FF900895BC0175
:1015E0008FE996E00E94C73008956091D804709109
:1015F000D9048091DA049091DB0420E030E040E1EE
:1016000052E40E94423620E030E044EB53E40E9472
:1016100074340E94A5360E94DC349B012550304072
:1016200037FF03C09B01215E3F4FA6E3B6E0F901FF
:10163000ED53FC4F80818C932F5F3F4F2432310557
:1016400014F020E030E0119686E0A134B80779F775
:101650001C9208952F923F924F925F926F927F92C9
:101660008F929F92AF92BF92CF92DF92EF92FF92B2
:101670000F931F93DF93CF9300D000D000D0CDB74E
:10168000DEB7182F662E2091CE043091CF042A3574
:10169000310530F0C9018D549F4F89359105E8F42B
:1016A00037FF02C02D543F4FC90137FF03C090954B
:1016B00081959F4F8A3191053CF0F4E48F2E912C57
:1016C000E9ED2E2E312C1DC00A975CF17BE3872EAD
:1016D000912C62ED262E312C20C02B35310514F0D3
:1016E000235B3040C90137FF03C0909581959F4F20
:1016F0008A31910554F056E5852E912C4CED242E1F
:10170000312C37E0A32EB12C15C00A9754F02DE4EC
:10171000822E912C94ED292E312C88E0A82EB12C0C
:1017200009C005E0802E912CB8E32B2E312CA9E0C6
:10173000AA2EB12C6091D0047091D104882777FD36
:101740008095982F0E940F3527EA32E94BE25CEB37
:101750000E9442360E94163720E030E040EA50E412
:101760000E94423620E030E040E951E40E944236D7
:101770000E94A53620E030E044E352E40E94A73303
:101780000E94DC34712EFEEBCF2EFFEFDF2E9B018B
:10179000442737FD4095542F29833A834B835C833C
:1017A000E6EA4E2EE4E05E2E4AEF5FEF240E351E91
:1017B0006091CE047091CF04882777FD8095982F93
:1017C0000E940F3525E33AEF4EE85CE30E94423673
:1017D0000E9416377B018C01B601882777FD809522
:1017E000982F0E940F359B01AC01C801B7010E94E0
:1017F00042367B018C0169817A818B819C810E94B8
:101800000F359B01AC01C801B7010E94A7330E94AC
:10181000DC349B01CB0101978A35910508F071C03A
:1018200062E170E00E947C378B012F5F3F4FAEEE8C
:10183000BFEF6A9FC0016B9F900D7A9F900D11249E
:10184000820F931F62E070E00E947C376D837E837D
:10185000E62CE01A4E2D4C5F86EA94E0672D0E943C
:101860000A0500D000D000D0EDB7FEB73196ADB775
:10187000BEB712965C924E92119720E031E033830E
:1018800022838D819E81880D991D958384830E947A
:10189000162A4DB75EB74A5F5F4F0FB6F8945EBF2A
:1018A0000FBE4DBF8D819E818A159B0554F104307A
:1018B00011053CF593E0E90EC201672D4E2D0E9403
:1018C0000A0500D000D000D0EDB7FEB73196ADB715
:1018D000BEB712965C924E92119720E031E03383AE
:1018E00022834D815E81420D531D558344830E94A6
:1018F000162A8DB79EB706960FB6F8949EBF0FBEF8
:101900008DBFACE0B0E0CA0EDB1E7394BEE4CB1614
:10191000D10409F04DCF26960FB6F894DEBF0FBE66
:10192000CDBFCF91DF911F910F91FF90EF90DF908E
:10193000CF90BF90AF909F908F907F906F905F906F
:101940004F903F902F900895823010F422E002C013
:10195000282F220F30E08DB79EB708970FB6F89466
:101960009EBF0FBE8DBFEDB7FEB7319686EA94E0FD
:10197000ADB7BEB712969C938E93119783E091E01A
:101980009383828322573F4F358324832F5F3F4FBA
:10199000378326830E94162A8DB79EB708960FB606
:1019A000F8949EBF0FBE8DBF0895CF93DF93AC0117
:1019B000E091E004F091E104209134063091350685
:1019C000C9018C599F4F8E179F071CF4EA0121977C
:1019D00009C024563040E217F30714F0EA0102C0B0
:1019E000EA012196842F90E0C817D90729F08FE9E2
:1019F00096E04C2F0E94CE30CE01DF91CF9108951A
:101A00000F931F930FE916E0C80163EF73E041E005
:101A10000E94CE30C80164EF73E043E10E94CE30F3
:101A2000C80165EF73E046E00E94CE30C80166EF62
:101A300073E040E10E94CE30C80167EF73E047E2F7
:101A40000E94CE30C80168EF73E048E80E94CE30B3
:101A5000C80169EF73E043E10E94CE301F910F91FE
:101A60000895CF92DF92EF92FF920F931F937C0124
:101A7000D62EC72E06EA14E0C8016E2D4D2D0E9409
:101A80007304C8010E944B0500D000D0EDB7FEB72B
:101A90001283018383E391E0948383830E94052A68
:101AA000EDB7FEB71283018383E291E094838383D1
:101AB0000E94052AEDB7FEB71283018383E191E00E
:101AC000948383830E94052AEDB7FEB712830183B6
:101AD00083E091E0948383830E94052AEDB7FEB7EB
:101AE0001283018384EF90E0948383830E94052A0C
:101AF0000F900F900F900F90C8010E942F05C70103
:101B000001966D2D7C2D0E942A0B1F910F91FF9045
:101B1000EF90DF90CF900895AF92BF92CF92DF9277
:101B2000EF92FF920F931F93B82EA62E0E94AF3113
:101B300028EE33E040E050E00E948F3779018A01BF
:101B4000A6EACA2EA4E0DA2EC6016B2D4A2D0E9409
:101B50007304C6010E944B05A090FE04B090FF04E0
:101B60008DB79EB744970FB6F8949EBF0FBE8DBF3A
:101B7000EDB7FEB73196ADB7BEB71296DC92CE92F6
:101B8000119788E091E09383828383EB90E09583C3
:101B90008483C7016CE370E00E947C37CB016CE367
:101BA00070E00E947C37978386832AE330E0318798
:101BB0002087C7016CE370E00E947C37938782879F
:101BC00085E690E095878487C5016CE370E00E940C
:101BD0006837CB016CE370E00E947C37978786877B
:101BE000318B208BC5016CE370E00E946837938BCA
:101BF000828B0E94162A8DB79EB744960FB6F89432
:101C00009EBF0FBE8DBFC6010E942F051F910F9171
:101C1000FF90EF90DF90CF90BF90AF900895EF923C
:101C2000FF920F931F93282F462FB6EAEB2EB4E0B6
:101C3000FB2EC701622F0E947304C7010E944B054F
:101C40008DB79EB70A970FB6F8949EBF0FBE8DBF93
:101C50000DB71EB70F5F1F4FEDB7FEB7F282E182DF
:101C600080E291E0F8019383828360910005709196
:101C70000105809102059091030520912B0630917A
:101C80002C0640912D0650912E060E944236F801F6
:101C9000648375838683978380EB90E09187808748
:101CA0000E94162A8DB79EB70A960FB6F8949EBF6B
:101CB0000FBE8DBFC7010E942F051F910F91FF908E
:101CC000EF9008958F929F92AF92BF92CF92DF9242
:101CD000EF92FF920F931F93E82EF62E06EA14E080
:101CE000C8016E2D4F2D0E947304C8010E944B0540
:101CF0008DB79EB70C970FB6F8949EBF0FBE8DBFE1
:101D0000EDB7FEB73196ADB7BEB712961C930E93E2
:101D1000119728E2822E21E0922E938282829DEEFC
:101D2000A92EB12CB582A4828091090590910A0553
:101D3000A0910B05B0910C0586839783A087B1878E
:101D400083EFC82ED12CD386C2860E94162A8DB767
:101D50009EB70C960FB6F8949EBF0FBE8DBFC801FC
:101D60000E942F05F394C8016E2D4F2D0E9473041D
:101D7000C8010E944B05ADB7BEB71C970FB6F894CB
:101D8000BEBF0FBEADBFEDB7FEB7319612961C9326
:101D90000E93119793828282B582A48280910D0561
:101DA00090910E05A0910F05B09110058683978341
:101DB000A087B187D386C2860E94162A8DB79EB7A8
:101DC0000C960FB6F8949EBF0FBE8DBFC8010E943F
:101DD0002F05F394C8016E2D4F2D0E947304C80186
:101DE0000E944B05ADB7BEB71C970FB6F894BEBFA7
:101DF0000FBEADBFEDB7FEB7319612961C930E9392
:101E0000119793828282B582A4828091110590916C
:101E10001205A0911305B091140586839783A087BE
:101E2000B187D386C2860E94162A8DB79EB70C96BC
:101E30000FB6F8949EBF0FBE8DBFC8010E942F053C
:101E40001F910F91FF90EF90DF90CF90BF90AF90D8
:101E50009F908F9008950F931F93282F462F06EA87
:101E600014E0C801622F0E947304C8010E944B0550
:101E70008DB79EB70A970FB6F8949EBF0FBE8DBF61
:101E8000EDB7FEB73196ADB7BEB712961C930E9361
:101E9000119782E391E09383828389EB90E09583AD
:101EA00084838091FC049091FD049783868382E86B
:101EB00090E0918780870E94162A8DB79EB70A9678
:101EC0000FB6F8949EBF0FBE8DBFC8010E942F05AC
:101ED0001F910F910895EF92FF920F931F93282F58
:101EE000462F36EAE32E34E0F32EC701622F0E941C
:101EF0007304C7010E944B058DB79EB70C970FB6B0
:101F0000F8949EBF0FBE8DBF0DB71EB70F5F1F4F5A
:101F1000EDB7FEB7F282E1828AE391E0F8019383A4
:101F2000828384EE90E0958384836091FA047091BB
:101F3000FB04882777FD8095982F0E940F352AE0B3
:101F400037ED43E25CE30E944236F8016683778313
:101F5000808791878FE890E0938782870E94162A76
:101F60008DB79EB70C960FB6F8949EBF0FBE8DBF6F
:101F7000C7010E942F051F910F91FF90EF900895C8
:101F80000F931F93282F462F06EA14E0C801622FF3
:101F90000E947304C8010E944B058DB79EB70C9731
:101FA0000FB6F8949EBF0FBE8DBFEDB7FEB731964A
:101FB000ADB7BEB712961C930E9311978AE391E0CA
:101FC0009383828382EE90E0958384838091F604EC
:101FD0009091F704A091F804B091F9048683978357
:101FE000A087B1878EE890E0938782870E94162AA7
:101FF0008DB79EB70C960FB6F8949EBF0FBE8DBFDF
:10200000C8010E942F051F910F9108950F931F93F0
:10201000282F462F86EA94E0622F0E94730486EAF6
:1020200094E00E944B058091DD04882319F424E498
:1020300031E057C0813019F428E431E052C08230D9
:1020400019F42CE431E04DC0833019F420E531E07F
:1020500048C0843019F424E531E043C0853019F4D8
:1020600028E531E03EC0863019F42CE531E039C076
:10207000873019F420E631E034C0883019F424E6C2
:1020800031E02FC0893019F428E631E02AC08A30C7
:1020900019F42CE631E025C08B3019F420E731E04B
:1020A00020C08C3019F424E731E01BC08D3019F4C6
:1020B00028E731E016C08E3019F42CE731E011C06A
:1020C0008F3019F420E831E00CC0803119F424E895
:1020D00031E007C0813119F028E831E002C029E879
:1020E00031E08DB79EB708970FB6F8949EBF0FBE2C
:1020F0008DBFEDB7FEB7319606EA14E0ADB7BEB7B7
:1021000012961C930E9311978DE891E0938382832E
:1021100080EE90E095838483378326830E94162A7D
:102120008DB79EB708960FB6F8949EBF0FBE8DBFB1
:10213000C8010E942F051F910F9108950F931F93BF
:10214000282F462F06EA14E0C801622F0E9473046C
:10215000C8010E944B058DB79EB70A970FB6F89439
:102160009EBF0FBE8DBFEDB7FEB73196ADB7BEB700
:1021700012961C930E93119782E991E093838283C8
:1021800087E890E0958384838091DE049091DF045A
:102190009783868385E290E0918780870E94162A44
:1021A0008DB79EB70A960FB6F8949EBF0FBE8DBF2F
:1021B000C8010E942F051F910F9108950F931F933F
:1021C000282F462F06EA14E0C801622F0E947304EC
:1021D000C8010E944B058DB79EB70A970FB6F894B9
:1021E0009EBF0FBE8DBFEDB7FEB73196ADB7BEB780
:1021F00012961C930E9311978CE991E0938382833E
:102200008091D0049091D1049583848380EB90E0F9
:102210009783868381EB90E0918780870E94162ABE
:102220008DB79EB70A960FB6F8949EBF0FBE8DBFAE
:10223000C8010E942F051F910F9108950F931F93BE
:10224000282F462F06EA14E0C801622F0E9473046B
:10225000C8010E944B058DB79EB70A970FB6F89438
:102260009EBF0FBE8DBFEDB7FEB73196ADB7BEB7FF
:1022700012961C930E9311978CE991E093838283BD
:102280008091CE049091CF049583848380EB90E07D
:102290009783868382EB90E0918780870E94162A3D
:1022A0008DB79EB70A960FB6F8949EBF0FBE8DBF2E
:1022B000C8010E942F051F910F9108950F931F933E
:1022C000282F462F06EA14E0C801622F0E947304EB
:1022D000C8010E944B058DB79EB70A970FB6F894B8
:1022E0009EBF0FBE8DBFEDB7FEB73196ADB7BEB77F
:1022F00012961C930E93119784EA91E09383828344
:1023000081EE90E0958384838091AC029091AD0240
:102310009783868385E290E0918780870E94162AC2
:102320008DB79EB70A960FB6F8949EBF0FBE8DBFAD
:10233000C8010E942F051F910F9108950F931F93BD
:10234000282F462F06EA14E0C801622F0E9473046A
:10235000C8010E944B058DB79EB70C970FB6F89435
:102360009EBF0FBE8DBFEDB7FEB73196ADB7BEB7FE
:1023700012961C930E9311978CEA91E093838283BB
:1023800086EB91E09583848380ED90E0978386834C
:1023900086E396E09187808781ED90E0938782873E
:1023A0000E94162A8DB79EB70C960FB6F8949EBF62
:1023B0000FBE8DBFC8010E942F051F910F91089578
:1023C0000F931F93282F462F06EA14E0C801622FAF
:1023D0000E947304C8010E944B058DB79EB70A97EF
:1023E0000FB6F8949EBF0FBE8DBFEDB7FEB7319606
:1023F000ADB7BEB712961C930E93119784EC91E083
:10240000938382838091D8049091D904A091DA04B7
:10241000B091DB0484839583A683B78380EB90E03F
:10242000918780870E94162A8DB79EB70A960FB6AD
:10243000F8949EBF0FBE8DBFC8010E942F051F914B
:102440000F9108950F931F93282F462F06EA14E04B
:10245000C801622F0E947304C8010E944B058DB70A
:102460009EB70C970FB6F8949EBF0FBE8DBFEDB709
:10247000FEB73196ADB7BEB712961C930E93119767
:102480008CEC91E09383828386E190E09583848352
:102490008091F2049091F304A091F404B091F504BA
:1024A00086839783A087B18788E890E093878287A7
:1024B0000E94162A8DB79EB70C960FB6F8949EBF51
:1024C0000FBE8DBFC8010E942F051F910F91089567
:1024D000CF92DF92EF92FF920F931F93CF93DF93F0
:1024E000282F462FC6EAD4E0CE01622F0E94730443
:1024F000CE010E944B056091420670914306809187
:1025000044069091450620912B0630912C0640916F
:102510002D0650912E060E9442366B017C0120E070
:1025200030E04AE754E40E9437361816D4F58DB7E8
:102530009EB70C970FB6F8949EBF0FBE8DBF0DB718
:102540001EB70F5F1F4FADB7BEB71296DC93CE9389
:1025500011978AE391E0F801938382838EEF90E0F4
:102560009583848360912F0670913006882777FDCC
:102570008095982F0E940F359B01AC01C701B601D1
:102580000E947434D80116966D937D938D939C931D
:102590001997809133061A968C931A971B961C9262
:1025A00021C08DB79EB70C970FB6F8949EBF0FBE93
:1025B0008DBFEDB7FEB73196ADB7BEB71296DC93BF
:1025C000CE93119786ED91E0938382838EEF90E016
:1025D00095838483C682D782E086F1868091320615
:1025E000828713860E94162AEDB7FEB73C960FB677
:1025F000F894FEBF0FBEEDBF86EA94E00E942F055F
:10260000DF91CF911F910F91FF90EF90DF90CF90CE
:102610000895EF92FF920F931F93282F462F56EAAB
:10262000E52E54E0F52EC701622F0E947304C70106
:102630000E944B058DB79EB70C970FB6F8949EBFBE
:102640000FBE8DBF0DB71EB70F5F1F4FEDB7FEB7A3
:10265000F282E1828CEC91E0F8019383828389EE2F
:1026600090E0958384836091EE047091EF048091F3
:10267000F0049091F10420912706309128064091B2
:10268000290650912A060E944236F8016683778314
:102690008087918780913106828713860E94162A4F
:1026A0008DB79EB70C960FB6F8949EBF0FBE8DBF28
:1026B000C7010E942F051F910F91FF90EF90089581
:1026C000EF92FF920F931F93282F462F66EAE62E74
:1026D00064E0F62EC701622F0E947304C7010E94B6
:1026E0004B058DB79EB70C970FB6F8949EBF0FBEE3
:1026F0008DBF0DB71EB70F5F1F4FEDB7FEB7F2824C
:10270000E18286ED91E0F8019383828386EE90E08A
:10271000958384836091EA047091EB048091EC04CA
:102720009091ED0420912B0630912C0640912D06BE
:1027300050912E060E944236F80166837783808787
:10274000918780913206828713860E94162A8DB760
:102750009EB70C960FB6F8949EBF0FBE8DBFC701F3
:102760000E942F051F910F91FF90EF900895EF9217
:10277000FF920F931F93282F462F76EAE72E74E0DF
:10278000F72EC701622F0E947304C7010E944B05F8
:102790008DB79EB70C970FB6F8949EBF0FBE8DBF36
:1027A0000DB71EB70F5F1F4FEDB7FEB7F282E18284
:1027B00086ED91E0F8019383828387EE90E0958324
:1027C00084836091040570910505882777FD8095C5
:1027D000982F0E940F3520912B0630912C064091A6
:1027E0002D0650912E060E944236F80166837783AB
:1027F0008087918780913206828713860E94162AED
:102800008DB79EB70C960FB6F8949EBF0FBE8DBFC6
:10281000C7010E942F051F910F91FF90EF9008951F
:102820000F931F93282F462F06EA14E0C801622F4A
:102830000E947304C8010E944B05809146060E94C5
:10284000A40CC8010E942F051F910F910895EF92CB
:10285000FF920F931F93282F462FE6EAEE2EE4E017
:10286000FE2EC701622F0E947304C7010E944B0510
:102870008DB79EB70C970FB6F8949EBF0FBE8DBF55
:102880000DB71EB70F5F1F4FEDB7FEB7F282E182A3
:1028900086ED91E0F801938382838FE190E0958348
:1028A0008483609147067091480680914906909113
:1028B0004A060E940F3520912B0630912C0640913C
:1028C0002D0650912E060E944236F80166837783CA
:1028D0008087918780913206828713860E94162A0C
:1028E0008DB79EB70C960FB6F8949EBF0FBE8DBFE6
:1028F000C7010E942F051F910F91FF90EF9008953F
:102900000F931F93282F462F06EA14E0C801622F69
:102910000E947304C8010E944B058DB79EB7409773
:102920000FB6F8949EBF0FBE8DBFEDB7FEB73196C0
:10293000ADB7BEB712961C930E93119780EE91E03F
:102940009383828383E890E0958384838091D40489
:102950009091D504A091D604B091D7048683978333
:10296000A087B18784E890E0938782878091E40410
:102970009091E504A091E604B091E70484879587DF
:10298000A687B7870E94162A8DB79EB740960FB6C6
:10299000F8949EBF0FBE8DBFC8010E942F051F91E6
:1029A0000F9108950F931F93282F462F86EA94E0E6
:1029B000622F0E94730486EA94E00E944B05809186
:1029C000E904282F30E0823030F4F4E0220F331F86
:1029D000FA95E1F702C02150304000D000D000D07D
:1029E000EDB7FEB7319606EA14E0ADB7BEB7129662
:1029F0001C930E93119780E091E09383828335833B
:102A000024830E94162A8DB79EB706960FB6F894B7
:102A10009EBF0FBE8DBFC8010E942F051F910F9151
:102A200008950F931F93282F462F06EA14E0C8013C
:102A3000622F0E947304C8010E944B058DB79EB798
:102A400008970FB6F8949EBF0FBE8DBFEDB7FEB7C7
:102A50003196ADB7BEB712961C930E93119782EFC5
:102A600091E0938382838FE090E0958384838091CB
:102A7000E804868317820E94162A8DB79EB70896AF
:102A80000FB6F8949EBF0FBE8DBFC8010E942F05E0
:102A90001F910F9108950F931F9306EA14E0C80148
:102AA00063E045E00E947304C8010E944B0500D01A
:102AB00000D0EDB7FEB71283018384E691E09483E2
:102AC00083830E94052AEDB7FEB71283018380E558
:102AD00091E0948383830E94052AEDB7FEB71283A9
:102AE000018389E491E0948383830E94052AEDB7F2
:102AF000FEB71283018383E491E0948383830E9471
:102B0000052A0F900F900F900F90C8010E942F057B
:102B10001F910F9108950F931F93282F462F06EAB8
:102B200014E0C801622F0E947304C8010E944B0583
:102B300000D000D0EDB7FEB7128301838BE791E0A0
:102B4000948383830E94052A0F900F900F900F901B
:102B5000C8010E942F051F910F910895EF92FF92D7
:102B60000F931F93CF93DF930E94AF3120915006B4
:102B7000309151064091520650915306261737075F
:102B80004807590708F08AC10E94AF316C507E4F48
:102B90008F4F9F4F6093500670935106809352065B
:102BA0009093530606EA14E0C8010E949805C801F4
:102BB00065E043E00E947304C8010E944B0500D009
:102BC00000D0EDB7FEB7128301838BED91E09483C3
:102BD00083830E94052A0F900F900F900F90809191
:102BE000340690913506892B31F080914B069091F7
:102BF0004C06892B81F48091E0049091E10490933C
:102C00003506809334068091E2049091E30490931A
:102C10004C0680934B062091E2043091E3044091EE
:102C20004B0650914C06C9018456904048175907ED
:102C300024F480914F068F5F08C02C593F4F241712
:102C400035072CF480914F06815080934F06809178
:102C50004F06181614F081E003C084301CF083E0A6
:102C600080934F0680914F06823009F462C0833012
:102C700009F4BEC0813009F00DC100D000D0C6EA11
:102C8000D4E0EDB7FEB7D283C18382ED91E09483A7
:102C900083830E94052A809125060F900F900F9044
:102CA0000F9080FF22C000D000D0EDB7FEB7D283D6
:102CB000C1838AEC91E0948383830E94052A8091EA
:102CC000340690913506845690400F900F900F90E7
:102CD0000F902091E0043091E104281739070CF09F
:102CE000D9C0809125068E7F21C000D000D0EDB7DD
:102CF000FEB7D283C18382EC91E0948383830E94E8
:102D0000052A80913406909135068C599F4F0F907B
:102D10000F900F900F902091E0043091E104821702
:102D200093070CF0B7C0809125068160809325063B
:102D3000B1C000D000D0C6EAD4E0EDB7FEB7D28370
:102D4000C18388EB91E0948383830E94052A0F90CE
:102D50000F900F900F9080914D06882301F100D0C5
:102D600000D0EDB7FEB7D283C1838EEA91E09483A1
:102D700083830E94052A80913406909135068456FB
:102D800090400F900F900F900F902091E0043091A1
:102D9000E104281739071CF510924D0620C000D019
:102DA00000D0EDB7FEB7D283C18381EA91E094836E
:102DB00083830E94052A80913406909135068C59B0
:102DC0009F4F0F900F900F900F902091E004309143
:102DD000E104821793071CF481E080934D068FE98C
:102DE00096E06BEF73E040914D060E94CE3052C0EA
:102DF00000D000D0A6EAEA2EA4E0FA2EEDB7FEB786
:102E0000F282E18280E991E0948383830E94052A23
:102E10008DB79EB708970FB6F8949EBF0FBE8DBFB3
:102E20000DB71EB70F5F1F4FEDB7FEB7F282E182FD
:102E300088EF91E0F8019383828360914E0670E001
:102E400080E090E00E940D3520E030E040E251E467
:102E50000E947434F801648375838683978386E7C0
:102E600090E09187808780E290E0938782870E943C
:102E7000162A8DB79EB70C960FB6F8949EBF0FBE5C
:102E80008DBF80914E0690E060E873E00E94D50C03
:102E900080934E0686EA94E00E942F05DF91CF9141
:102EA0001F910F91FF90EF9008952F923F924F92B4
:102EB0005F926F927F928F929F92AF92BF92CF92CA
:102EC000DF92EF92FF920F931F93DF93CF93CDB7D3
:102ED000DEB72B970FB6F894DEBF0FBECDBF888745
:102EE00069870E94AF3120915D0630915E06409166
:102EF0005F0650916006261737074807590708F004
:102F000069C1809161068823C9F08093AE02109256
:102F1000610680E092E090936306809362060E94CF
:102F2000AF316C507E4F8F4F9F4F60935D06709313
:102F30005E0680935F069093600607C18091AE02A3
:102F4000282E33242091DC042F83009162061091F7
:102F500063063091C90439838091E9048E8390918E
:102F600054069D83E09016056090F6047090F70477
:102F70008090F8049090F90490914E064090AC0235
:102F80005090AD0280915506A82FB0E0BC83AB8372
:102F9000B0915606BA83F09015053B862A86A92E75
:102FA000BB24CC24DD24EA85FB853196FB87EA87A8
:102FB00037972CF021E030E03B872A871CC08A85B8
:102FC0009B858330910539F1843091053CF4813043
:102FD000910589F0029709F07FC015C0AA85BB85CD
:102FE000A530B10509F44EC0A530B10504F116971E
:102FF00009F072C058C0BF81B23008F06DC00DE05A
:1030000012E081E070C0E981E33009F465C00AE1B3
:1030100012E082E068C0FE81F23008F05DC02D81D0
:10302000222309F459C007E212E083E05CC031E0DA
:103030003E1598F0C601B5010E940D3520E030E044
:1030400040E251E40E9474349B01AC01C401B3011D
:103050000E946D3488230CF03FC004E312E083E04B
:10306000E81649F094E0E91649F0A2E0EA1641F4C6
:1030700001E412E005C00EE412E002C00BE512E02C
:1030800084E031C0EB81FC814E165F062CF5FDE932
:103090004F16FFEF5F0601F12A812223E9F408E6CB
:1030A00012E085E020C03F813230B0F481E08F151E
:1030B00098F493E0F91649F0A4E0FA1649F0B2E06A
:1030C000FB1651F405E712E005C001E812E002C06A
:1030D0000EE812E086E007C0EA85FB85E215F305FD
:1030E00009F061CF60C0109363060093620680937D
:1030F000610681E0809357060E94AF3168517C4F92
:103100008F4F9F4F60935D0670935E0680935F06BE
:10311000909360060E94AF316056704F8F4F9F4F63
:103120006093590670935A0680935B0690935C06F1
:1031300080915806882321F086EA94E00E94980541
:103140001092580602C01092570606EA14E0C80111
:10315000688549850E947304C8010E944B0500D010
:1031600000D000D0EDB7FEB73196ADB7BEB712961E
:103170001C930E9311978BE992E093838283809145
:10318000620690916306958384830E94162AEDB7A8
:10319000FEB736960FB6F894FEBF0FBEEDBFC8015E
:1031A0000E942F0517C010936306009362061092C9
:1031B00061060E94AF312091590630915A06409124
:1031C0005B0650915C06261737074807590708F435
:1031D000BACFBBCF2B960FB6F894DEBF0FBECDBFD4
:1031E000CF91DF911F910F91FF90EF90DF90CF90E3
:1031F000BF90AF909F908F907F906F905F904F9017
:103200003F902F900895EF92FF920F931F9380911C
:103210006406843009F056C09091DD04943008F0C3
:1032200027C180916D068917A1F190936D060E94C8
:10323000AF316093690670936A0680936B06909332
:103240006C0690916D068091AF02981711F58091F0
:103250005806813091F0813018F08230B1F413C0FB
:1032600011E0109358060E94AF31615375478040BA
:10327000904030F41093650608C082E080935806B1
:103280001092650602C01092580686EA94E00E94E9
:1032900098050E94AF312091690630916A064091ED
:1032A0006B0650916C06621B730B840B950B615D72
:1032B00077408040904008F4DBC08091DD0480932B
:1032C000AF02D6C0853029F48091A4029091A50266
:1032D00014C0863029F48091A6029091A7020DC0F7
:1032E000873029F48091A8029091A90206C0883005
:1032F00041F48091AA029091AB029093680680936A
:1033000067068091660620916706309168068823DB
:1033100009F04AC0C901895097408F5A9440C8F4B7
:103320000E94AF31615375478040904020F481E0A6
:10333000809365060CC080916506882341F48091D6
:103340005706882321F486EA94E00E94980582E0DB
:1033500028C044E0203B340768F480915806882355
:1033600049F01092650686EA94E00E949805109252
:1033700058067EC0205B34402955324008F078C0A2
:1033800080915806813009F473C0809157068823D4
:1033900009F06EC01092650686EA94E00E949805D6
:1033A00081E08093580664C0215B344008F460C01B
:1033B0000E94AF31615375478040904008F041C092
:1033C000809165068823E9F5E0906906F0906A0629
:1033D00000916B0610916C0688EE93E0A0E0B0E0DF
:1033E000E80EF91E0A1F1B1F0E94AF31E616F706F2
:1033F00008071907E8F581E08093650617C0109269
:10340000650686EA94E00E9498058091580682300D
:1034100019F41092580603C08F5F8093580680916C
:103420005806823018F082E0809358060E94AF312F
:103430006093690670936A0680936B0690936C069E
:1034400017C0E0906906F0906A0600916B06109133
:103450006C0688EE93E0A0E0B0E0E80EF91E0A1FCB
:103460001B1F0E94AF31E616F7060807190738F24E
:103470001F910F91FF90EF90089580916406843022
:1034800010F00E94031980916506882319F00E94AC
:10349000AE1508958091090480FF08C060916F0403
:1034A00080916D0490E070E00E945517809158065D
:1034B000823008F0FDC1A82FB0E0FD01ED5FFB4FA9
:1034C000808185FF0BC0FD01E15EFB4F6081A35E43
:1034D000BB4F8C9190E070E00E94111580915806CE
:1034E000A82FB0E0FD01ED5FFB4F808186FF0BC090
:1034F000FD01ED5DFB4F6081AF5DBB4F8C9190E0B6
:1035000070E00E94D21480915406882309F43FC0D1
:1035100080915806A82FB0E0FD01ED5FFB4F808140
:1035200087FF0BC0FD01E95DFB4F6081AB5DBB4FC9
:103530008C9190E070E00E94801480915806A82F32
:10354000B0E0FD01EB5FFB4F808184FF0BC0FD010C
:10355000E15CFB4F6081A35CBB4F8C9190E070E01D
:103560000E94271480915806A82FB0E0FD01EB5F60
:10357000FB4F808183FF0BC0FD01E55CFB4F608149
:10358000A75CBB4F8C9190E070E00E94101480917A
:103590005806A82FB0E0FD01E95FFB4F808187FF4F
:1035A0000BC0FD01E95AFB4F6081AB5ABB4F8C91B8
:1035B00090E070E00E94B71380915806A82FB0E009
:1035C000FD01E75FFB4F808183FF0BC0FD01E958E0
:1035D000FB4F6081AB58BB4F8C9190E070E00E9434
:1035E000221280915406882309F46EC08091E90468
:1035F000823008F469C080915806A82FB0E0FD0120
:10360000E55FFB4F808182FF0BC0FD01ED57FB4F53
:103610006081AF57BB4F8C9190E070E00E946812C0
:1036200080915806A82FB0E0FD01E95FFB4F808133
:1036300082FF0BC0FD01ED5AFB4F6081AF5ABB4FBB
:103640008C9190E070E00E94601380915806A82F42
:10365000B0E0FD01E95FFB4F808183FF0BC0FD01FE
:10366000E55AFB4F6081A75ABB4F8C9190E070E008
:103670000E94091380915806A82FB0E0FD01EB5F6E
:10368000FB4F808181FF0BC0FD01ED5CFB4F608132
:10369000AF5CBB4F8C9190E070E00E94E011809194
:1036A0005806A82FB0E0FD01EB5FFB4F808180FF43
:1036B0000BC0FD01E15DFB4F6081A35DBB4F8C91B1
:1036C00090E070E00E949E1180915806A82FB0E013
:1036D000FD01E75FFB4F808186FF0BC0FD01E158D4
:1036E000FB4F6081A358BB4F8C9190E070E00E942B
:1036F0005E1180915806A82FB0E0FD01ED5FFB4FF1
:10370000808182FF0BC0FD01E95EFB4F6081AB5EF3
:10371000BB4F8C9190E070E00E941E118091580682
:10372000A82FB0E0FD01ED5FFB4F808181FF0BC052
:10373000FD01ED5EFB4F6081AF5EBB4F8C9190E071
:1037400070E00E94DE1080915806A82FB0E0FD01C5
:10375000E95FFB4F808184FF0BC0FD01ED59FB4FFA
:103760006081AF59BB4F8C9190E070E00E949E1039
:1037700080915806A82FB0E0FD01E95FFB4F8081E2
:1037800085FF0BC0FD01E959FB4F6081AB59BB4F71
:103790008C9190E070E00E94061080915806A82F4E
:1037A000B0E0FD01ED5FFB4F808183FF0BC0FD01A9
:1037B000E55EFB4F6081A75EBB4F8C9190E070E0AF
:1037C0000E94C00F80915806A82FB0E0FD01E95F6C
:1037D000FB4F808180FF0BC0FD01E15BFB4F6081EF
:1037E000A35BBB4F8C9190E070E00E946B0F8091C7
:1037F0005806A82FB0E0FD01ED5FFB4F808184FFEC
:103800000BC0FD01E55DFB4F6081A75DBB4F8C9157
:1038100090E070E00E942B0F80915806A82FB0E036
:10382000FD01E55FFB4F808181FF18C080914D064F
:10383000FD01EB57FB4F813049F4A957BB4F6C9109
:10384000808190E070E00E940F0E08C0A957BB4F26
:103850006C91808190E070E00E94620E8091580629
:10386000A82FB0E0FD01EB5FFB4F808187FF0BC00D
:10387000FD01E55BFB4F6081A75BBB4F8C9190E046
:1038800070E00E948C0D80915806A82FB0E0FD01D9
:10389000E95FFB4F808186FF0BC0FD01E559FB4FBF
:1038A0006081A759BB4F8C9190E070E00E94310D70
:1038B000089586EA94E00E9498050E944B150E94A4
:1038C0000A0A0895CF93DF93EC0186EA94E00E9400
:1038D0006F04C817D9073CF086EA94E00E9464049C
:1038E000892B09F42397CE01DF91CF910895EF92B0
:1038F000FF920F931F93CF93DF930091580610E030
:103900008AEF90E0089F7001099FF00C189FF00C5F
:103910001124C7010E94EF0AF801ED5FFB4F8823D5
:1039200019F08081816002C080818E7F80838091C8
:103930005806C82FD0E0C70102960E94EF0AC35F65
:10394000DB4F888380915806C82FD0E0C7010496CA
:103950000E94EF0A90E00E94621CC15FDB4F8883E7
:103960000091580610E0C70188569F4F0E94EF0A49
:10397000F801ED5FFB4F882319F08081806102C060
:1039800080818F7E808380915806C82FD0E0C70148
:1039900086569F4F0E94EF0AC75DDB4F8883809158
:1039A0005806C82FD0E0C70184569F4F0E94EF0AE7
:1039B00090E00E94621CC55DDB4F88830091580631
:1039C00010E0C70106960E94EF0AF801ED5FFB4F79
:1039D000882319F08081826002C080818D7F80837E
:1039E00080915806C82FD0E0C70108960E94EF0AC0
:1039F000CF5EDB4F888380915806C82FD0E0C70187
:103A00000A960E94EF0A90E00E94621CCD5EDB4F96
:103A100088830091580610E0C7010C960E94EF0AB7
:103A2000F801ED5FFB4F882319F08081846002C0AC
:103A300080818B7F808380915806C82FD0E0C7019A
:103A40000E960E94EF0ACB5EDB4F8883809158066A
:103A5000C82FD0E0C70140960E94EF0A90E00E9474
:103A6000621CC95EDB4F88830091580610E0C701D5
:103A700042960E94EF0AF801ED5FFB4F882319F090
:103A80008081886002C08081877F80838091580612
:103A9000C82FD0E0C70144960E94EF0AC75EDB4FF3
:103AA000888380915806C82FD0E0C70146960E94AF
:103AB000EF0A90E00E94621CC55EDB4F8883009194
:103AC000580610E0C7014E960E94EF0AF801ED5F1C
:103AD000FB4F882319F08081806202C080818F7D36
:103AE000808380915806C82FD0E0C70180960E943D
:103AF000EF0AC35EDB4F888380915806C82FD0E061
:103B0000C70182960E94EF0A90E00E94621CC15E8B
:103B1000DB4F88830091580610E0C70184960E940D
:103B2000EF0AF801ED5FFB4F882319F08081806474
:103B300002C080818F7B808380915806C82FD0E09F
:103B4000C70186960E94EF0ACF5DDB4F8883809184
:103B50005806C82FD0E0C70188960E94EF0A90E06F
:103B60000E94621CCD5DDB4F88830091580610E0F7
:103B7000C7018A960E94EF0AF801ED5FFB4F882388
:103B800019F08081806802C080818F778083809166
:103B90005806C82FD0E0C7018C960E94EF0ACB5D73
:103BA000DB4F888380915806C82FD0E0C7018E96DE
:103BB0000E94EF0A90E00E94621CC95DDB4F88837F
:103BC0000091580610E0C701C0960E94EF0AF80164
:103BD000EB5FFB4F882319F08081816002C08081F8
:103BE0008E7F808380915806C82FD0E0C701C2968F
:103BF0000E94EF0AC35DDB4F888380915806C82F6F
:103C0000D0E0C701C4960E94EF0A90E00E94621CB7
:103C1000C15DDB4F88830091580610E0C701C6964E
:103C20000E94EF0AF801EB5FFB4F882319F08081B7
:103C3000826002C080818D7F808380915806C82F6A
:103C4000D0E0C701C8960E94EF0ACF5CDB4F8883A3
:103C500080915806C82FD0E0C701CA960E94EF0A8B
:103C600090E00E94621CCD5CDB4F88830091580677
:103C700010E0C701CC960E94EF0AF801EB5FFB4F02
:103C8000882319F08081846002C080818B7F8083CB
:103C900080915806C82FD0E0C701CE960E94EF0A47
:103CA000CB5CDB4F888380915806C82FD0E0C701DA
:103CB000805C9F4F0E94EF0A90E00E94621CC95CEA
:103CC000DB4F88830091580610E0C701885B9F4F47
:103CD0000E94EF0AF801EB5FFB4F882319F0808107
:103CE000806102C080818F7E808380915806C82FBA
:103CF000D0E0C701865B9F4F0E94EF0AC35CDB4F99
:103D0000888380915806C82FD0E0C701845B9F4FFD
:103D10000E94EF0A90E00E94621CC15CDB4F888326
:103D20000091580610E0C7018E5B9F4F0E94EF0A7A
:103D3000F801EB5FFB4F882319F08081886002C097
:103D40008081877F808380915806C82FD0E0C7018B
:103D50008C5B9F4F0E94EF0AC75CDB4F888380918A
:103D60005806C82FD0E0C7018A5B9F4F0E94EF0A18
:103D700090E00E94621CC55CDB4F8883009158066E
:103D800010E0C701805B9F4F0E94EF0AF801EB5FD4
:103D9000FB4F882319F08081806202C080818F7D73
:103DA000808380915806C82FD0E0C7018E5A9F4F5C
:103DB0000E94EF0ACF5BDB4F888380915806C82FA3
:103DC000D0E0C7018C5A9F4F0E94EF0A90E00E94FA
:103DD000621CCD5BDB4F88830091580610E0C70161
:103DE0008A5A9F4F0E94EF0AF801EB5FFB4F88232E
:103DF00019F08081806402C080818F7B80838091F4
:103E00005806C82FD0E0C701885A9F4F0E94EF0A7A
:103E1000CB5BDB4F888380915806C82FD0E0C70169
:103E2000865A9F4F0E94EF0A90E00E94621CC95B75
:103E3000DB4F88830091580610E0C70182569F4FE0
:103E40000E94EF0AF801EB5FFB4F882319F0808195
:103E5000806802C080818F77808380915806C82F48
:103E6000D0E0C70180569F4F0E94EF0AC75BDB4F2F
:103E7000888380915806C82FD0E0C7018E559F4F88
:103E80000E94EF0A90E00E94621CC55BDB4F8883B2
:103E90000091580610E0C7018E599F4F0E94EF0A0B
:103EA000F801E95FFB4F882319F08081816002C02F
:103EB00080818E7F808380915806C82FD0E0C70113
:103EC0008C599F4F0E94EF0AC35BDB4F8883809120
:103ED0005806C82FD0E0C7018A599F4F0E94EF0AA9
:103EE00090E00E94621CC15BDB4F88830091580602
:103EF00010E0C70182599F4F0E94EF0AF801E95F65
:103F0000FB4F882319F08081846002C080818B7F01
:103F1000808380915806C82FD0E0C70180599F4FF9
:103F20000E94EF0ACF5ADB4F888380915806C82F32
:103F3000D0E0C7018E589F4F0E94EF0A90E00E9488
:103F4000621CCD5ADB4F88830091580610E0C701F0
:103F500084579F4F0E94EF0AF801E95FFB4F8823C7
:103F600019F08081806802C080818F778083809182
:103F70005806C82FD0E0C70182579F4F0E94EF0A12
:103F8000CB5ADB4F888380915806C82FD0E0C701F9
:103F900080579F4F0E94EF0A90E00E94621CC95A0E
:103FA000DB4F88830091580610E0C7018E569F4F63
:103FB0000E94EF0AF801E95FFB4F882319F0808126
:103FC000826002C080818D7F808380915806C82FD7
:103FD000D0E0C7018C569F4F0E94EF0AC35ADB4FB7
:103FE000888380915806C82FD0E0C7018A569F4F1A
:103FF0000E94EF0A90E00E94621CC15ADB4F888346
:104000000091580610E0C7018C589F4F0E94EF0A9C
:10401000F801E95FFB4F882319F08081886002C0B6
:104020008081877F808380915806C82FD0E0C701A8
:104030008A589F4F0E94EF0AC75ADB4F88838091AE
:104040005806C82FD0E0C70188589F4F0E94EF0A3A
:1040500090E00E94621CC55ADB4F8883009158068D
:1040600010E0C70186589F4F0E94EF0AF801E95FF0
:10407000FB4F882319F08081806102C080818F7E90
:10408000808380915806C82FD0E0C70184589F4F85
:104090000E94EF0ACF59DB4F888380915806C82FC2
:1040A000D0E0C70182589F4F0E94EF0A90E00E9423
:1040B000621CCD59DB4F88830091580610E0C70180
:1040C00080589F4F0E94EF0AF801E95FFB4F882359
:1040D00019F08081806202C080818F7D8083809111
:1040E0005806C82FD0E0C7018E579F4F0E94EF0A95
:1040F000CB59DB4F888380915806C82FD0E0C70189
:104100008C579F4F0E94EF0A90E00E94621CC95991
:10411000DB4F88830091580610E0C7018A579F4FF4
:104120000E94EF0AF801E95FFB4F882319F08081B4
:10413000806402C080818F7B808380915806C82F65
:10414000D0E0C70188579F4F0E94EF0AC759DB4F45
:10415000888380915806C82FD0E0C70186579F4FAB
:104160000E94EF0A90E00E94621CC559DB4F8883D1
:104170000091580610E0C7018C559F4F0E94EF0A2E
:10418000F801E75FFB4F882319F08081816002C04E
:1041900080818E7F808380915806C82FD0E0C70130
:1041A0008A559F4F0E94EF0AC359DB4F8883809145
:1041B0005806C82FD0E0C70188559F4F0E94EF0ACC
:1041C00090E00E94621CC159DB4F88830091580621
:1041D00010E0C70180559F4F0E94EF0AF801E75F8A
:1041E000FB4F882319F08081846002C080818B7F1F
:1041F000808380915806C82FD0E0C7018E549F4F0E
:104200000E94EF0ACF58DB4F888380915806C82F51
:10421000D0E0C7018C549F4F0E94EF0A90E00E94AB
:10422000621CCD58DB4F88830091580610E0C7010F
:104230008A549F4F0E94EF0AF801E75FFB4F8823E3
:1042400019F08081886002C08081877F808380919F
:104250005806C82FD0E0C70188549F4F0E94EF0A2C
:10426000CB58DB4F888380915806C82FD0E0C70118
:1042700086549F4F0E94EF0A90E00E94621CC9582A
:10428000DB4F88830091580610E0C70184549F4F8C
:104290000E94EF0AF801E75FFB4F882319F0808145
:1042A000806102C080818F7E808380915806C82FF4
:1042B000D0E0C70182549F4F0E94EF0AC758DB4FDE
:1042C000888380915806C82FD0E0C70180549F4F43
:1042D0000E94EF0A90E00E94621CC558DB4F888361
:1042E0000091580610E0C701845A9F4F0E94EF0AC0
:1042F000F801E75FFB4F882319F08081806402C0DA
:1043000080818F7B808380915806C82FD0E0C701C1
:10431000825A9F4F0E94EF0AC358DB4F88838091D7
:104320005806C82FD0E0C701805A9F4F0E94EF0A5D
:1043300090E00E94621CC158DB4F888300915806B0
:1043400010E0C70180529F4F0E94EF0AF801E55F1D
:10435000FB4F882319F08081846002C080818B7FAD
:10436000808380915806C82FD0E0C7018E519F4F9F
:104370000E94EF0ACF57DB4F888380915806C82FE1
:10438000D0E0C7018C519F4F0E94EF0A90E00E943D
:10439000621CCD57DB4F88830091580610E0C7019F
:1043A0008C529F4F0E94EF0AF801E55FFB4F882374
:1043B00019F08081826002C080818D7F808380912E
:1043C0005806C82FD0E0C7018A529F4F0E94EF0ABB
:1043D000CB57DB4F888380915806C82FD0E0C701A8
:1043E00088529F4F0E94EF0A90E00E94621CC957BA
:1043F000DB4F8883DF91CF911F910F91FF90EF905A
:1044000008954F925F927F928F929F92AF92BF9248
:10441000CF92DF92EF92FF920F931F93DF93CF9390
:10442000CDB7DEB7C854D0400FB6F894DEBF0FBE8C
:10443000CDBF06EA14E0C8010E949805C80166E0F5
:1044400049E00E947304C8010E944B0500D000D0CF
:10445000EDB7FEB71283018386E092E094838383F5
:104460000E94052A0F900F900F900F90C8010E9494
:104470002F0500D000D009E814E0EDB7FEB7128395
:10448000018386EF91E0948383830E94052A4BEE9B
:10449000442E41E0542EEE24FF24CC24DD240F9042
:1044A0000F900F900F90702E012F39E0A32EB12C9A
:1044B000AC0EBD1E4E010894811C911C89E894E04D
:1044C0000E94B92A982F8D3031F08D30DCF1805365
:1044D0008230C0F530C01830A1F59981892F805302
:1044E000823078F5913311F490E801C090E08A8130
:1044F000813309F4905C8B81813309F4905E8C8167
:10450000813309F4905F8D81813309F4985F8E8146
:10451000813309F49C5F8F81813309F49E5F888524
:10452000813309F49F5FF501EE0DFF1D9083089420
:10453000E11CF11C06C0F401E10FF11D90831F5F27
:1045400001C010E0F0E4EF16F104C9F486EA94E04B
:10455000B601A5010E9483040894C11CD11C00D09F
:1045600000D0EDB7FEB771820283548243820E946D
:10457000052AEE24FF240F900F900F900F90FFEF6D
:10458000CF16D10409F00CF499CFC85BDF4F0FB6FA
:10459000F894DEBF0FBECDBFCF91DF911F910F9179
:1045A000FF90EF90DF90CF90BF90AF909F908F9053
:1045B0007F905F904F900895DF92EF92FF920F935C
:1045C0001F93DF93CF93CDB7DEB72A970FB6F8943A
:1045D000DEBF0FBECDBF63E0E62EF12CEC0EFD1E5C
:1045E00053E0D52EF6C30E94AF3160527E44804026
:1045F0009040C8F40E94AF316958734180409040A8
:1046000090F01A3011F01D3031F4809121068F5F47
:104610008093210602C010922106809121068330EA
:1046200011F40E940122812F67E175E00E94F506D6
:10463000882311F400E0C7C380911B0590911C05ED
:10464000A0911D05B0911E05863E46EA940746E2FC
:10465000A4074DE7B40709F48EC2873E56EA9507D2
:1046600056E2A5075DE7B50708F0EFC08832EEE532
:104670009E07E2EDAE07E4E2BE0709F427C28932E5
:10468000FEE59F07F2EDAF07F4E2BF0708F06AC04E
:1046900088392CE292072AE1A20726E1B20709F441
:1046A0001EC289393CE293073AE1A30736E1B3071A
:1046B00040F586314AEA940747E3A4074BE0B40784
:1046C00009F404C287315AEA950757E3A5075BE06E
:1046D000B50738F48E5F9B4CA74CB94009F069C30D
:1046E00060C38430FAE99F07F7EDAF07FEE0BF072C
:1046F00009F4ECC18259934AAC4EB44109F059C354
:10470000E5C184373BEE93073AE7A3073BE1B307E4
:1047100009F4DCC185374BEE94074AE7A4074BE167
:10472000B40780F480355FED95075DEEA50758E18D
:10473000B50709F40BC38E5C9844A745BA4109F04C
:1047400038C319C28434FBED9F07F0E7AF07FDE1E2
:10475000BF0709F426C3825D924CA248BE4109F00E
:1047600028C3BDC1883536EB93073DEFA3073AE474
:10477000B30709F4CDC2893546EB94074DEFA40782
:104780004AE4B40788F5863E55ED95075AEDA5072E
:1047900053E3B50709F448C1873EE5ED9E07EAED0E
:1047A000AE07E3E3BE0780F48E37F9EA9F07FBE527
:1047B000AF07F6E2BF0709F492C182559342A649BA
:1047C000B64209F0F6C254C2883F3CEA93073EEE77
:1047D000A30734E3B30709F4E4C2865A9E40A2411A
:1047E000B84409F0E6C27DC280365BED95075BE315
:1047F000A5075EE6B50709F469C18136EBED9E07B2
:10480000EBE3AE07EEE6BE0780F4823EF5E59F07D8
:10481000FCE9AF07F6E6BF0709F48AC28C5E99434C
:10482000A647BB4609F0C5C2BCC28A3B37EC93071A
:1048300031E2A30734E7B30709F4F6C08A57974C6F
:10484000A94DBB4709F0B5C2ACC28A3B54E89507F5
:1048500055E2A5075EEBB50709F46AC28B3BE4E8B5
:104860009E07E5E2AE07EEEBBE0708F06AC08E37A2
:10487000F2E19F07FAE6AF07FBE9BF0709F426C19B
:104880008F3722E192072AE6A2072BE9B20740F50B
:1048900082353AEE930730E8A3073AE8B30709F404
:1048A00015C183354AEE940740E8A4074AE8B407E7
:1048B00038F486549340A24CB54809F07AC271C2CC
:1048C0008C38E5E89E07E7EAAE07E8E9BE0709F499
:1048D00052C18A569E42A246B94909F06AC201C233
:1048E00080322EE4920729EAA20721EBB20709F4ED
:1048F0001FC281323EE4930739EAA30731EBB307C5
:1049000080F48A3746EF940741EFA4074DE9B407D6
:1049100009F431C18E5F964BA942B54A09F049C2EC
:104920002AC18A38E7EF9E07E7ECAE07E8EBBE073F
:1049300009F4D5C0845A9040AB49BA4B09F039C24A
:1049400030C2843629ED920720EEA20727EDB20788
:1049500009F46AC0853639ED930730EEA30737EDC9
:10496000B30788F586384BE3940740EAA40744EC84
:10497000B40709F4DDC187385BE3950750EAA50762
:1049800054ECB50780F48C36E8E69E07E3E4AE0706
:10499000E2ECBE0709F45CC180589447A041B44CD6
:1049A00009F007C29CC084352DE292072FEFA207C1
:1049B00025ECB20709F48AC086599543A840B24D48
:1049C00009F0F7C155C18E344DE594074EE3A407B5
:1049D00043EEB40709F47AC08F345DE595075EE3D2
:1049E000A50753EEB50780F48437E7E39E07E4EDAF
:1049F000AE07EEEDBE0709F49BC1865B9342A34A66
:104A0000B24E09F0D6C1B7C0823920E7920726E836
:104A1000A2072BEFB20709F4C4C1825F9D4EA442E6
:104A2000BD4F09F0C6C18DC10E94AF316093CA0469
:104A30007093CB048093CC049093CD04D092C9049E
:104A400087E195E060E170E00E94C9080E94DC34D3
:104A50007093CF046093CE0487E195E064E170E049
:104A60000E94C9080E94DC347093D1046093D00482
:104A700087E195E068E170E00E94C9080E94DC349B
:104A80008B017093D3046093D2046091D40470912D
:104A9000D5048091D6049091D70420E030E040E026
:104AA00050E00E946D34882379F4B801882777FD9F
:104AB0008095982F0E940F356093D8047093D90485
:104AC0008093DA049093DB0401E074C180912105A6
:104AD0008093DC04809122058093DD046AC187E124
:104AE00095E060E070E00E94C90820E030E048EC0A
:104AF00052E40E9442360E94DC347093DF046093DB
:104B0000DE04693C710520F01092DF041092DE048F
:104B100080913B0590913C059093E1048093E004E3
:104B200080913D0590913E059093E3048093E204CB
:104B300080914105909142059093A5028093A40233
:104B400080914505909146059093A7028093A60217
:104B500080914705909148059093A9028093A802FF
:104B60008091490590914A059A8389839093AB027D
:104B70008093AA021EC16091210570912205809147
:104B80002305909124050E940F3520E836E948E17D
:104B90005BE40E9474346093D4047093D5048093D2
:104BA000D6049093D70460912505709126058091D5
:104BB000270590912805D7016C9311967C93119746
:104BC00012968C93129713969C930E940F3520E8AF
:104BD00036E948E15BE40E9474346093E404709326
:104BE000E5048093E6049093E70480914605809362
:104BF000E804809145058093E90487E195E060E150
:104C000070E00E94C9086093D8047093D90480931F
:104C1000DA049093DB0487E195E068E070E00E949D
:104C2000C9086093EA047093EB048093EC049093BA
:104C3000ED0487E195E064E170E00E94C9086093AB
:104C4000EE047093EF048093F0049093F104B1C0EC
:104C500087E195E068E070E00E94C9089058609391
:104C6000F2047093F3048093F4049093F504A1C0CC
:104C700087E195E060E070E00E94C9086093F60467
:104C80007093F7048093F8049093F90487E195E01A
:104C900064E070E00E94C90820E030E048EC52E493
:104CA0000E9442360E94DC347093FB046093FA0445
:104CB00087E195E064E170E00E94C9080E94DC345D
:104CC0007093FD046093FC0487E195E068E170E077
:104CD0000E94C9080E94DC347093FF046093FE04B4
:104CE00068C087E195E064E070E00E94C9080E9416
:104CF000DC34882777FD8095982F0E940F356093CC
:104D0000000570930105809302059093030551C03F
:104D100087E195E068E070E00E94C9080E94DC34F9
:104D2000709561957F4F709305056093040541C0B0
:104D30008091810580930605809182058093070507
:104D400038C0809121058093080533C087E195E044
:104D500060E070E00E94C9086093090570930A053D
:104D600080930B0590930C0587E195E064E070E07B
:104D70000E94C90860930D0570930E0580930F057E
:104D80009093100587E195E068E070E00E94C90803
:104D90006093110570931205809313059093140589
:104DA00008C080912D058093150580913205809370
:104DB000160500E080911805823229F487E195E01C
:104DC00063E20E94E1098EEB90E00E94163200231C
:104DD00031F589E894E00E94892A18161906F4F43E
:104DE00089E894E00E94B92A182F8091C904882389
:104DF00009F019CCF8CB1092C90401E0802F90E0A3
:104E00002A960FB6F894DEBF0FBECDBFCF91DF91CB
:104E10001F910F91FF90EF90DF90089500E0209197
:104E2000CA043091CB044091CC045091CD04205F52
:104E3000384D4F4F5F4F2F83388749875A870E94DD
:104E4000AF312F81388549855A852617370748079E
:104E5000590788F2D3CFEF92FF920F931F9380915F
:104E60005606882351F083E00E944B3364E070E0E3
:104E70000E947C37609326063CC083E00E944B333F
:104E8000AA2797FDA095BA2FBC01CD010E940F352E
:104E90002DEC3CEC4CE45EE30E94423620E030E036
:104EA00040E85EE30E9442367B018C016091260659
:104EB00070E0882777FD8095982F0E940F352DECA4
:104EC0003CEC4CE45FE30E9442369B01AC01C8011C
:104ED000B7010E94A7330E94E13420917106621746
:104EE00030F030917006262F361708F4232F2093C8
:104EF00026061F910F91FF90EF90089583E00E9486
:104F0000483308951F93CF93DF9385E090E06CE0E2
:104F100070E00E948B1568EE73E080E090E00E94E4
:104F2000BD3189E894E00E94062BC0E0D0E010E09B
:104F3000CE016DE171E00E947C37892BA9F41F5EE0
:104F400086EA94E0612F4CE00E94730486EA94E0C4
:104F50000E944B0586EA94E06EEE0E947B0586EA8D
:104F600094E00E942F05105161E070E080E090E035
:104F70000E94BD31219687E0C13DD807C9F6DF9177
:104F8000CF911F91089586E061E00E94F432089568
:104F90000F931F9386E061E00E94B53209E814E0A8
:104FA000C80140E051EE60E070E00E94272A1093B3
:104FB000A1060093A0060E94C32786EA94E00E94FF
:104FC000D1050E94591C64EF71E080E090E00E94DE
:104FD000BD3183EF93E00E94EF0A813011F00E940F
:104FE000000D0E94600A1092580607C00E94771CAC
:104FF000809158068F5F80935806809158068230C2
:10500000A8F3109258060E9482270E947E2788EB00
:1050100094E069E979E224E630E040E050E000E025
:105020000E94DA3086EA94E00E94980588EB94E0CA
:105030000E9440311F910F9108952F923F924F92FD
:105040005F926F927F928F929F92AF92BF92CF9218
:10505000DF92EF92FF920F931F93DF93CF9300D0D5
:1050600000D0CDB7DEB780915406882309F4E1C0A3
:10507000E0907906F0907A0600917B0610917C060C
:10508000C801B7019F7725E33AEF4EE85CE30E9441
:1050900042360E94713469837A838B839C83C80172
:1050A000B7012091D4043091D5044091D604509199
:1050B000D7040E94A6331B012C019F7720EC3BE60E
:1050C00049ED57E40E9442365B016C0160917D0618
:1050D00070917E0680917F06909180062091E40475
:1050E0003091E5044091E6045091E7040E94A63314
:1050F0003B014C019F7720EC3BE649ED57E40E94D1
:10510000423629813A814B815C810E9442367B0183
:105110008C01C601B501A60195010E9442365B01D2
:105120006C01C801B701A80197010E9442369B019A
:10513000AC01C601B5010E94A7330E94C9360E9486
:10514000DC34609347067093480680934906909339
:105150004A0660E070E080E89FE329813A814B8154
:105160005C810E9474349B01AC01C201B1010E94B8
:10517000423697FA909497F89094A40193010E9474
:105180001A3420EE3EE245E652E40E94423620E028
:1051900030E044EB52E40E94A7330E94DC349B01D0
:1051A000AC0197FF04C028593E4F4F4F5F4FCA01D3
:1051B000B901645B70408040904097FF06C0CA010F
:1051C000B9016C547F4F8F4F9F4F0E940F35209134
:1051D000D8043091D9044091DA045091DB040E9444
:1051E000A6330E94DC3497FF04C068597E4F8F4F6E
:1051F0009F4F0E940F3520E030E044EB53E40E94C3
:10520000743420E030E040E851E40E9442360E94CD
:10521000A53620E030E040E85FE30E94A7330E941B
:10522000E13460934606613108F46CC01092460682
:1052300069C08091E904823008F464C08091E80478
:10524000853008F45FC0A09081068DE18A1508F4CE
:1052500059C0E090EA04F090EB040091EC04109146
:10526000ED0460918206709183068091840690918E
:105270008506A80197010E94A6339F7720E030E0C1
:1052800040E05FE30E94373618165CF41092810606
:10529000E0928206F09283060093840610938506BE
:1052A00031C08A2D8F5F809381068E3159F58091B0
:1052B000D4049091D504A091D604B091D7048093E2
:1052C000790690937A06A0937B06B0937C06809132
:1052D000E4049091E504A091E604B091E704809382
:1052E0007D0690937E06A0937F06B0938006E092A1
:1052F0008606F0928706009388061093890681E05F
:10530000809354060F900F900F900F90CF91DF91E4
:105310001F910F91FF90EF90DF90CF90BF90AF90D3
:105320009F908F907F906F905F904F903F902F90C5
:105330000895CF92DF92EF92FF920F931F930E94F6
:105340002B2780912606282F30E03093AD02209342
:10535000AC0280915606882359F50091710610E041
:10536000201B310BB901882777FD8095982F0E946B
:105370000F356B017C016091700670E0601B710B52
:10538000882777FD8095982F0E940F359B01AC01EF
:10539000C701B6010E94743420E030E048EC52E4CA
:1053A0000E9442360E94DC347093AD026093AC02DE
:1053B0008091AC029091AD028D599F4F34F48DE9EC
:1053C0009FEF9093AD028093AC020E9452080E941E
:1053D000F50A86EA94E00E941D280E943D1A1F915A
:1053E0000F91FF90EF90DF90CF9008950E94DC2204
:1053F000892B19F00E949929089588EB94E00E9466
:10540000283108958FEF9FE70895DF93CF93CDB7AD
:10541000DEB7FE0139968D819E8161E04F8158850E
:105420009F010E94A62CCF91DF910895DF93CF9327
:10543000CDB7DEB7FE0139968D819E8160E04F8148
:1054400058859F010E94A62CCF91DF9108950F935C
:105450001F93DC01ED91FC910288F389E02D20E09F
:1054600030E000E010E009951F910F9108958F92B0
:10547000AF92CF92EF92FF920F931F93DF93CF9350
:10548000CDB7DEB7FC011382128288EE93E0A0E074
:10549000B0E084839583A683B7838BEE93E09183FA
:1054A00080835587448737872687118B008BF38A43
:1054B000E28AC48AA58A868A70E0CB0123E0880F3D
:1054C000991F2A95E1F79C012257394F308F278B7E
:1054D0008A56994F928F818F81E090E002C0880FA9
:1054E000991F6A95E2F720919E06282B20939E062D
:1054F000CF0140E051EE60E070E00E94272ACF919A
:10550000DF911F910F91FF90EF90CF90AF908F9010
:105510000895FC01838D882319F42FEF3FEF0DC010
:105520000788F08DE02D2081318182819381281BB5
:10553000390B8481958128233923C9010895FC0101
:10554000838D882319F42FEF3FEF11C0018CF28D6A
:10555000E02D2081318182819381281B390B209598
:10556000309584819581282339232F5F3F4FC901CE
:105570000895FC01838D882361F0A789B08D2D915A
:105580003C91119712968D919C911397281739078A
:1055900021F44FEF5FEFCA01089512968D919C910F
:1055A00013971696ED91FC911797E80FF91F40811C
:1055B00012968D919C911397019614962D913C9182
:1055C00015978223932313969C938E93129750E002
:1055D000E2CFFC01838D882351F00788F08DE02D08
:1055E00020813181828193812817390721F42FEF9F
:1055F0003FEFC9010895828193810680F781E02DF4
:10560000E80FF91F8081282F30E0F3CFDC01579697
:10561000ED91FC9158978281938191838083599673
:10562000ED91FC915A9780819181938382830895B3
:10563000DC015B968C915B978823A9F15996ED91DB
:10564000FC915A97208131812F5F3F4F8481958152
:10565000282339235C968C915C97882329F08281DA
:10566000938128173907F9F0828193812817390728
:10567000D9F3808191810680F781E02DE80FF91F31
:1056800060835996ED91FC915A973183208352960D
:10569000ED91FC915397808156969C91892B808344
:1056A00021E030E002C020E030E0C9010895CF934E
:1056B000DF93EC011B821A828A819B819983888304
:1056C0001D821C828E819F81009721F00E94C5035C
:1056D0001F821E82DF91CF9108950F931F938C013B
:1056E000DC015296ED91FC915397208156968C9156
:1056F000569755969C915597892B80958223808348
:1057000057968D919C9158970E94572BF801818D47
:10571000928D0E94572BD8015B961C921F910F917E
:1057200008950F931F93CF93DF938C01FC01138295
:105730001282828193819183808341E0A1E0B0E075
:1057400001C04F5FFD01042E02C0EE0FFF1F0A943F
:10575000E2F79B0182E06130780710F020E032E050
:10576000E217F30770F3C1E0D0E002C0CC0FDD1FF9
:105770004A95E2F72197F8012681378121153105F5
:1057800041F0848195818C179D0789F0C9010E94A1
:10579000C503F801D583C483CE0101960E941B0383
:1057A0009C01F8019783868380E0232B09F081E038
:1057B000DF91CF911F910F910895AF92BF92CF9239
:1057C000DF92EF92FF920F931F93CF93DF937C01B1
:1057D0005A016B01E901DC015B968C915B97882390
:1057E000F1F02115310539F45796ED91FC91589758
:1057F000C481D58121960115110549F4D701599627
:10580000ED91FC915A97048115810F5F1F4FD701CD
:10581000ED91FC910088F189E02DC7010995F70110
:105820008789908D209711F4C0E8D0E0BE010E94D6
:10583000912B882381F0D70159968D919C915A978D
:105840000115110511F400E110E0B8010E94912B3F
:10585000882309F04DC0D701ED91FC910088F189B2
:10586000E02DC701099567C0D7015096ED91FC91D5
:105870005197B0E0AB16B1EEBB06B0E0CB06B0E09E
:10588000DB0609F454C081E090E0D70154960C90F7
:1058900002C0880F991F0A94E2F7808360E079E0E4
:1058A0008DE390E0A60195010E94B1372150304070
:1058B00040405040CA01B90122E030E040E050E0F1
:1058C0000E94B137D7011C96ED91FC911D97308352
:1058D0001E96ED91FC911F972083D7015296ED9172
:1058E000FC915397808155969C91892B808323C08E
:1058F000D7015996ED91FC915A97138212828281B9
:105900009381918380835796ED91FC9158971382F0
:105910001282828193819183808381E05B968C9354
:105920001A141B041C041D040CF49ECFD6CF108245
:1059300020E130E0C7CFDF91CF911F910F91FF9011
:10594000EF90DF90CF90BF90AF9008952F923F924D
:105950004F925F926F927F928F929F92AF92BF927F
:10596000CF92DF92EF92FF920F931F93DF93CF932B
:10597000CDB7DEB764970FB6F894DEBF0FBECDBFCC
:105980003C01688B5A8B498B69011C01AE014F5F4A
:105990005F4F5C8B4B8BE989FA89488940FD6591A3
:1059A00040FF6191FA8BE98B662309F4D7C3653216
:1059B00049F440FD859140FF8191FA8BE98B853256
:1059C000B1F40CC06A3051F4D301ED91FC91019017
:1059D000F081E02DC1016DE009956AE0D301ED9100
:1059E000FC910190F081E02DC1010995D4CF982F51
:1059F00010E0882499241032B0F49B3269F09C3274
:105A000028F4903251F0933271F40BC09D3239F08A
:105A1000903349F4116028C01260146025C01860EA
:105A200023C0106121C017FD2BC0892F80538A30FD
:105A300078F416FF06C0BAE09B9E902C1124980EB5
:105A400013C0EAE08E9E802C1124880E10620CC0D8
:105A50009E3221F416FD82C3106406C09C3611F4F8
:105A6000106802C0983661F4E989FA89488940FDD6
:105A7000959140FF9191FA8BE98B992309F0BBCF67
:105A8000892F8554833020F4812F8061905E07C078
:105A9000892F8556833008F0E6C1812F8F7E86FDE1
:105AA00002C076E0972E6FE3F62EF822953619F4B1
:105AB00050E4F52A07C0963619F480E8F82A02C0A7
:105AC00091109A94F7FE0BC09BE3991520F427E000
:105AD0005CE3B52E0DC0B92CB39427E009C0A7E054
:105AE000A91520F447E0942E27E001C0292DBB24FE
:105AF000F6013496FD87EC87D6016D917D918D91ED
:105B00009C91AE014F5F5F4F0B2D0E9443026C01D1
:105B10000981E02FF0E0FF87EE8700FF05C0FE85DA
:105B2000F3FD02C01DE209C0F1FE02C01BE205C088
:105B3000F2FC02C010E001C010E28E859F858C70DF
:105B40009070892B09F444C0112311F483E001C043
:105B500084E0881510F088240EC0881AF3FC0BC06E
:105B6000D301ED91FC910190F081E02DC10160E243
:105B700009958A94A9F7112349F0D301ED91FC917D
:105B80000190F081E02DC101612F0995BE85B3FF21
:105B900003C00FE013E012C003E113E00FC0E114F3
:105BA000F10409F06052D301ED91FC910190F08174
:105BB000E02DC10109950F5F1F4F05C0EF2CFF2499
:105BC000B0E1EB22FF24F8016491662341F748C15C
:105BD000F7FE13C0BC0CFE85F4FF04C08A8181333C
:105BE00009F4BA941B141CF0BB24B3942DC048E0F4
:105BF0004B1550F538E0B32E27C0F6FC25C0892D93
:105C000090E08C159D054CF05CEFC5165FEFD50656
:105C100024F080E8F82A01C09A94992049F0E2E043
:105C2000F0E0EC0FFD1FE90DF11D80818033A1F341
:105C3000F7FE0AC0B92CB394892D90E0C816D90696
:105C400014F0992401C09C18F7FC03C025E030E053
:105C500009C01C141D041CF021E030E003C09601B3
:105C60002F5F3F4F112311F02F5F3F4F992029F0F5
:105C7000892D90E00196280F391F882D90E0281774
:105C8000390714F0882401C0821A4F2C5524C20110
:105C900089709070892B59F00CC0D301ED91FC9163
:105CA0000190F081E02DC10160E209958A9488207D
:105CB000A1F7112349F0D301ED91FC910190F081FE
:105CC000E02DC101612F099543FE0BC00CC0D3012B
:105CD000ED91FC910190F081E02DC10160E3099507
:105CE0008A948820A1F7F7FE51C08601D7FE02C032
:105CF00000E010E076010894E11CF11CE01AF10AC2
:105D0000E1E0F0E0EC0FFD1FEE0EFF1E26014B1848
:105D10005108892D90E0AA24BB24A81AB90AFFEFE4
:105D20000F3F1F0749F4D301ED91FC910190F081E1
:105D3000E02DC1016EE20995C016D10634F040167F
:105D400051061CF4F701608101C060E3015010406E
:105D50000894E11CF11C0A151B054CF0D301ED91D0
:105D6000FC910190F081E02DC1010995D8CF0C156F
:105D70001D0541F48A81863320F4853319F4BE85EC
:105D8000B4FF61E3D301ED91FC9165C06A81613399
:105D900009F00F7ED301ED91FC910190F081E02D8F
:105DA000C10109959920E1F0D301ED91FC91019099
:105DB000F081E02DC1016EE2099512E0E1E0F0E032
:105DC000EC0FFD1FE10FF11D60811F5FD301ED910D
:105DD000FC910190F081E02DC10109959A9471F731
:105DE000D301ED91FC910190F081E02D44FC02C0C3
:105DF00065E601C065E4C1010995D7FC05C0C11481
:105E0000D10441F404FF06C0D094C194D108D394C6
:105E10006DE201C06BE2D301ED91FC910190F08144
:105E2000E02DC101099560E305C06F5FE6EFFFEF6C
:105E3000CE0EDF1EFAE0CF16D104BCF7D301ED91F0
:105E4000FC910190F081E02DC1010995D301ED9104
:105E5000FC916C2D605D0190F081E02DC1010995F0
:105E6000CC84DD8478C1933631F0933799F0933543
:105E700009F061C023C0F601808189835E01089426
:105E8000A11CB11C42E050E0C40ED51E21E0E22E60
:105E9000F12C12C0D601AD90BC9016FD03C06FEF7F
:105EA0007FEF02C0692D70E0E2E0F0E0CE0EDF1E71
:105EB000C5010E9428047C011F7713C0D601AD9054
:105EC000BC9016FD03C06FEF7FEF02C0692D70E03C
:105ED000E2E0F0E0CE0EDF1EC5010E941D047C0151
:105EE000106813FF0BC023C0D301ED91FC9101900A
:105EF000F081E02DC10160E209958A94882D90E03F
:105F0000E816F90688F313C0F50117FD659117FF30
:105F100061915F01D301ED91FC910190F081E02D41
:105F2000C101099581108A940894E108F108E114EF
:105F3000F10451F710C1943611F0993699F517FF15
:105F40000AC0F601208131814281538184E090E0D2
:105F5000C80ED91E0CC0D6018D919C919C0144277E
:105F600037FD4095542FE2E0F0E0CE0EDF1E9FE6B5
:105F7000F92EF12257FF09C0509540953095219593
:105F80003F4F4F4F5F4FF0E8FF2ACA01B901AE0102
:105F90004F5F5F4F2AE030E00E94E501E82E4B8919
:105FA000E41A41C0953721F41F7E2AE030E01CC07E
:105FB000197F9F3661F0903720F4983509F0CEC0F4
:105FC0000FC0903739F0983709F0C8C004C028E0F6
:105FD00030E00AC0106114FD146020E130E004C01C
:105FE00014FD166020E132E017FF08C0D6016D9164
:105FF0007D918D919C91E4E0F0E008C0D6018D91F7
:106000009C91BC0180E090E0E2E0F0E0CE0EDF1E6B
:10601000AE014F5F5F4F0E94E501E82EFB89EF1A4A
:106020008FE7F82EF122F6FE0BC04EEFF422E914B2
:1060300038F4F4FE07C0F2FC05C05FEEF52202C0A2
:106040001E2D01C0192DF4FE0DC0FE01EE0DF11D37
:106050008081803319F489EEF82208C01F5FF2FEB8
:1060600005C003C08F2D867809F01F5F0F2DF3FC4C
:1060700018C0F0FE13C0181510F09E2C0FC09E2CF7
:10608000980C911A182D0AC0D301ED91FC91019042
:10609000F081E02DC10160E209951F5F1815A0F3A2
:1060A00004C0181510F4811A01C0882404FF17C019
:1060B000D301ED91FC910190F081E02DC10160E3ED
:1060C000099502FF29C0D301ED91FC910190F08167
:1060D000E02D01FD02C068E712C068E510C0802F06
:1060E0008678D1F001FF02C06BE201C060E2F7FCEC
:1060F0006DE2D301ED91FC910190F081E02DC101A1
:1061000009950AC0D301ED91FC910190F081E02D39
:10611000C10160E309959A94E914A0F3EA94D301CC
:10612000ED91FC91A1E0B0E0AC0FBD1FAE0DB11D33
:106130000190F081E02DC1016C910995EE2071F77D
:106140000AC0D301ED91FC910190F081E02DC101D5
:1061500060E209958A948820A1F71DCC64960FB659
:10616000F894DEBF0FBECDBFCF91DF911F910F918D
:10617000FF90EF90DF90CF90BF90AF909F908F9067
:106180007F906F905F904F903F902F900895F99976
:10619000FECF72BD61BDF89A80B50895F999FECF22
:1061A0001FBA72BD61BD40BD0FB6F894FA9AF99A54
:1061B0000FBE08950F93FC016115710511F480E085
:1061C00011C02183328343835483728761870170B6
:1061D000000F000F000F8081877F802B82608B7FF4
:1061E000808381E00F910895CF93DF93EC010E94AB
:1061F000AF319B01AC018D819E81AF81B88528179D
:1062000039074A075B0728F4888184FD02C060E0F3
:106210000DC089819A81AB81BC81820F931FA41F1D
:10622000B51F8D839E83AF83B88761E0222757FD1A
:106230002395332744275527922F91709295907F6D
:1062400088818F7E892B8883862FDF91CF91089557
:10625000CF93DF93EC01888182FF0FC0CE010E94B3
:10626000F430882351F0E985FA85309709F00995D3
:10627000888183FF02C08B7F8883DF91CF9108954F
:10628000CF93DF93EC0189859A85892BE1F0898191
:106290009A81AB81BC810097A105B105A1F00E9454
:1062A000AF3129813A814B815C81260F371F481F0E
:1062B000591F2D833E834F835887888184608F7E4A
:1062C000888381E001C080E0DF91CF9108951F9223
:1062D0000F920FB60F9211242F933F938F939F939A
:1062E000AF93BF938091A6069091A706A091A806B0
:1062F000B091A9063091AA060196A11DB11D232FC8
:106300002D5F2D3720F02D570196A11DB11D209333
:10631000AA068093A6069093A706A093A806B0931A
:10632000A9068091A2069091A306A091A406B0911F
:10633000A5060196A11DB11D8093A2069093A30608
:10634000A093A406B093A506BF91AF919F918F91A2
:106350003F912F910F900FBE0F901F9018958FB700
:10636000F8942091A6063091A7064091A806509176
:10637000A9068FBFB901CA0108959B01AC017FB77F
:10638000F8948091A2069091A306A091A406B091E2
:10639000A50666B5A89B05C06F3F19F00196A11D23
:1063A000B11D7FBFBA2FA92F982F8827860F911D67
:1063B000A11DB11D62E0880F991FAA1FBB1F6A951E
:1063C000D1F7BC012DC0FFB7F8948091A20690913F
:1063D000A306A091A406B091A506E6B5A89B05C0AA
:1063E000EF3F19F00196A11DB11DFFBFBA2FA92FD4
:1063F000982F88278E0F911DA11DB11DE2E0880FF7
:10640000991FAA1FBB1FEA95D1F7861B970B885EC1
:106410009340C8F2215030404040504068517C4F7A
:10642000211531054105510571F60895019739F09F
:10643000880F991F880F991F02970197F1F7089508
:10644000789484B5826084BD84B5816084BD85B54F
:10645000826085BD85B5816085BDEEE6F0E0808116
:1064600081608083E1E8F0E0108280818260808337
:10647000808181608083E0E8F0E0808181608083BA
:10648000E1EBF0E0808184608083E0EBF0E08081EC
:1064900081608083EAE7F0E080818460808380818E
:1064A0008260808380818160808380818068808336
:1064B0001092C10008951F920F920FB60F921124EF
:1064C0002F933F934F935F936F937F938F939F93FC
:1064D000AF93BF93EF93FF938091AB069091AC067F
:1064E000892B29F0E091AB06F091AC060995FF915C
:1064F000EF91BF91AF919F918F917F916F915F913C
:106500004F913F912F910F900FBE0F901F901895B4
:106510001F920F920FB60F9211242F933F934F9318
:106520005F936F937F938F939F93AF93BF93EF93FB
:10653000FF938091AD069091AE06892B29F0E091F2
:10654000AD06F091AE060995FF91EF91BF91AF9125
:106550009F918F917F916F915F914F913F912F917B
:106560000F900FBE0F901F901895CF93DF93482F79
:1065700050E0CA01875B9C4FFC0134914B5C5C4F3F
:10658000FA018491882369F190E0880F991FFC013A
:10659000E95EFC4FA591B491FC01EF5DFC4FC59104
:1065A000D491662351F42FB7F8948C91932F909542
:1065B00089238C93888189230BC0623061F42FB7C3
:1065C000F8948C91932F909589238C938881832BB9
:1065D00088832FBF06C09FB7F8948C91832B8C9330
:1065E0009FBFDF91CF910895482F50E0CA01835A91
:1065F0009C4FFC012491CA01875B9C4FFC01949144
:106600004B5C5C4FFA013491332309F440C02223E0
:1066100051F1233071F0243028F42130A1F02230E0
:1066200011F514C02630B1F02730C1F02430D9F470
:1066300004C0809180008F7703C0809180008F7D9F
:106640008093800010C084B58F7702C084B58F7DA1
:1066500084BD09C08091B0008F7703C08091B000E5
:106660008F7D8093B000E32FF0E0EE0FFF1FEF5D12
:10667000FC4FA591B4912FB7F894662321F48C9127
:106680009095892302C08C91892B8C932FBF0895FC
:106690008093B0020895982F8E3008F09E50977026
:1066A0008091B0028295880F880F807C892B80931F
:1066B0007C0080917A00806480937A0080917A00D7
:1066C00086FDFCCF2091780040917900942F80E0E6
:1066D00030E0282B392BC9010895CF92DF92EF9239
:1066E000FF920F931F93CF93DF937C016B018A017D
:1066F000C0E0D0E00FC0D6016D916D01D701ED91E2
:10670000FC910190F081E02DC7010995C80FD91FB8
:10671000015010400115110571F7CE01DF91CF91A5
:106720001F910F91FF90EF90DF90CF900895CF933E
:10673000DF930E9420320E94C827C0E0D0E00E9470
:10674000F6292097E1F30E940000F9CF5058BB27AB
:10675000AA270ED041C201D230F006D220F031F487
:106760009F3F11F41EF4C0C10EF4E095E7FBB6C1E3
:10677000E92F54D280F3BA1762077307840795078D
:1067800018F071F49EF56CC20EF4E0950B2EBA2F42
:10679000A02D0B01B90190010C01CA01A001112427
:1067A000FF27591B99F0593F50F4503E68F11A16D3
:1067B000F040A22F232F342F4427585FF3CF469564
:1067C00037952795A795F0405395C9F77EF41F1686
:1067D000BA0B620B730B840BBAF09150A1F0FF0F50
:1067E000BB1F661F771F881FC2F70EC0BA0F621F3C
:1067F000731F841F48F4879577956795B795F7952C
:106800009E3F08F0B3CF9395880F08F09927EE0FBD
:10681000979587950895A1D158F080E891E009F403
:106820009EEFA2D128F040E851E059F45EEF09C094
:106830005BC116C2E92FE078F1D168F3092E052A71
:10684000C1F3261737074807590738F00E2E07F807
:10685000E02569F0E025E0640AC0EF6307F80094E2
:1068600007FADB01B9019D01DC01CA01AD01EF931B
:106870004AD0B2D10AD05F91552331F02BED3FE0E1
:1068800049E450FD49EC63CF0895DF93DD27B92F2C
:10689000BF7740E85FE31616170648075B0710F45A
:1068A000D92FE9D19F938F937F936F93BCD2E8E662
:1068B000F0E01DD191D12F913F914F915F91EED199
:1068C000DD2349F09058A2EA2AED3FE049EC5FE36E
:1068D000D0785D274DDFDF917FC1DCD008F481E007
:1068E00008954AD1E39589C10CD076C13DD140F0DD
:1068F00034D130F021F45F3F19F0F0C05111B1C133
:10690000F3C08CD198F39923C9F35523B1F3951BA8
:10691000550BBB27AA2762177307840738F09F5FC0
:106920005F4F220F331F441FAA1FA9F333D00E2E2F
:106930003AF0E0E830D091505040E695001CCAF79C
:1069400029D0FE2F27D0660F771F881FBB1F261761
:1069500037074807AB07B0E809F0BB0B802DBF0134
:10696000FF2793585F4F2AF09E3F510568F0B6C04D
:1069700078C15F3FECF3983EDCF386957795679599
:10698000B795F7959F5FC9F7880F911D96958795E5
:1069900097F90895E1E0660F771F881FBB1F621704
:1069A00073078407BA0720F0621B730B840BBA0BC2
:1069B000EE1F88F7E095089504D06894B11151C195
:1069C000089534D188F09F5790F0B92F9927B75187
:1069D000A0F0D1F0660F771F881F991F1AF0BA95A3
:1069E000C9F712C0B13081F03BD1B1E0089538C190
:1069F000672F782F8827B85F39F0B93FCCF3869599
:106A000077956795B395D9F73EF4909580957095F5
:106A100061957F4F8F4F9F4F0895E89409C097FB72
:106A20003EF490958095709561957F4F8F4F9F4F65
:106A30009923A9F0F92F96E9BB279395F6958795A9
:106A400077956795B795F111F8CFFAF4BB0F11F46C
:106A500060FF1BC06F5F7F4F8F4F9F4F16C0882313
:106A600011F096E911C0772321F09EE8872F762F49
:106A700005C0662371F096E8862F70E060E02AF08A
:106A80009A95660F771F881FDAF7880F9695879576
:106A900097F90895990F0008550FAA0BE0E8FEEF4B
:106AA00016161706E807F907C0F012161306E407D2
:106AB000F50798F0621B730B840B950B39F40A26CB
:106AC00061F0232B242B252B21F408950A2609F4A9
:106AD000A140A6958FEF811D811D089597F99F67AD
:106AE00080E870E060E008959FEF80EC0895DF9308
:106AF000CF931F930F93FF92EF92DF927B018C0154
:106B0000689405C0DA2EEF01C9D0FE01E894A59182
:106B10002591359145915591AEF3EF0129DEFE01A6
:106B20009701A801DA9479F7DF90EF90FF900F9129
:106B30001F91CF91DF9108959F938F937F936F93D0
:106B4000FF93EF939B01AC019DD0EF91FF91CFDFBD
:106B50002F913F914F915F9195C000240A94161692
:106B6000170618060906089500240A94121613063B
:106B7000140605060895B8CF59D0E8F3E894EFEF6E
:106B8000BB273FE048EC5FE76B3D73078407950741
:106B900008F1FF279F57B25A6A4D7F40894CF04059
:106BA00032F4BE556542704F8643FF4F0894EE1F86
:106BB000915030F0BB0F661F771F881FFF1FEBCF70
:106BC0009EE7882332F0BB0F661F771F881F9A95B8
:106BD000C1F79395E09565C1092E0394000C11F45B
:106BE000882352F0BB0F40F4BF2B11F460FF04C0A8
:106BF0006F5F7F4F8F4F9F4F0895EF93E0FF06C069
:106C0000A2EA2AED3FE049EC5FEBB2DDE5DF0F9051
:106C1000039401FC9058E5E9F0E08ECF57FD9058C1
:106C2000440F551F59F05F3F71F04795880F97FB50
:106C3000991F61F09F3F79F087950895121613060A
:106C40001406551FF2CF4695F1DF08C01616170639
:106C50001806991FF1CF869571056105089408956E
:106C6000E894BB2766277727CB0197F9089512DFB1
:106C700008F48FEF08959B01AC0160E070E080E8BC
:106C80009FE332CE0BD0A8CF68DF28F06DDF18F07D
:106C9000952309F023CF28CF1124E3CFBFDFA0F342
:106CA000959FD1F3950F50E0551F629FF001729FA1
:106CB000BB27F00DB11D639FAA27F00DB11DAA1FC0
:106CC000649F6627B00DA11D661F829F2227B00D0D
:106CD000A11D621F739FB00DA11D621F839FA00D98
:106CE000611D221F749F3327A00D611D231F849FE8
:106CF000600D211D822F762F6A2F11249F5750403F
:106D00008AF0E1F088234AF0EE0FFF1FBB1F661FD9
:106D1000771F881F91505040A9F79E3F510570F092
:106D2000DDCE9FCF5F3FECF3983EDCF38695779501
:106D30006795B795F795E7959F5FC1F7FE2B880F8D
:106D4000911D9695879597F9089570DFE0F09E372D
:106D5000D8F09639B8F49E3848F4672F782F8827F2
:106D6000985FF9CF86957795679593959539D0F388
:106D7000B62FB1706B0F711D811D20F4879577952B
:106D80006795939573C08DC06CCF11F40EF4ACCEA3
:106D900088C04CDFD0F39923D9F3CEF39F57550B1E
:106DA00087FF8FD056959795B0E020F4660F771F38
:106DB000881FBB1F1F930F9300249001A001800127
:106DC000F001A0E80E0F1F1F0A1E511D601B710B62
:106DD0008009B50B48F4600F711F801DB51F0E1B95
:106DE0001F0B0A0A510907C02E0F3F1F4A1F0E0F23
:106DF0001F1F0A1E511D660F771F881FBB1FA695F8
:106E0000F795E795F8F60617170708065B07211DA3
:106E1000311D411D0F911F91B901842F9158880F89
:106E20009695879508959B01AC012CCFDF93D92FC0
:106E3000A3DEE695D7952AED3FE049E45FE3B33A58
:106E40006207730784079507D7952AF0A2EA49ECF1
:106E500090688EDCC1DEE3EBF0E06EDEDD0F0BF060
:106E60000ADFDD0F0BF49058DF910895882371F449
:106E7000772321F09850872B762F07C0662311F4D3
:106E800099270DC09051862B70E060E02AF09A950A
:106E9000660F771F881FDAF7880F9695879597F901
:106EA00008959F3F49F0915028F48695779567950E
:106EB000B7959F5F80389F4F880F9695879597F974
:106EC000089591505040660F771F881FD2F708959C
:106ED000AA1BBB1B51E107C0AA1FBB1FA617B70700
:106EE00010F0A61BB70B881F991F5A95A9F780951C
:106EF0009095BC01CD01089597FB092E07260AD075
:106F000077FD04D0E5DF06D000201AF47095619576
:106F10007F4F0895F6F7909581959F4F0895A1E2D0
:106F20001A2EAA1BBB1BFD010DC0AA1FBB1FEE1F03
:106F3000FF1FA217B307E407F50720F0A21BB30B4E
:106F4000E40BF50B661F771F881F991F1A9469F7CA
:106F500060957095809590959B01AC01BD01CF0126
:106F6000089597FB092E05260ED057FD04D0D7DFD4
:106F70000AD0001C38F450954095309521953F4F2C
:106F80004F4F5F4F0895F6F79095809570956195F6
:106F90007F4F8F4F9F4F0895EE0FFF1F0590F49185
:086FA000E02D0994F894FFCFE5
:106FA800256300256325630025632532692563254C
:106FB8003032697C256325326925632530326900C2
:106FC80025352E3066256300256325312E35662547
:106FD80063002563253569256300256325352E3231
:106FE800662563006D616E0073743100737432003E
:106FF800737433007374340073743500737436001B
:1070080070682000636C200076722000686C200095
:1070180061702000727462006C616E0070702000F4
:10702800706F69006163200000617420002563258A
:107038007300256325332E306925630025346925BF
:1070480063256300256325336925630025737C2543
:1070580063257325630020C0C0C0C0C0C7C0C0C0BE
:10706800C0C0200025342E306625630025632533F3
:107078002E3066256300256325352E30662563008E
:1070880025632531312E36667C25632531312E3630
:10709800660025632532690025332E316625630095
:1070A80020202020202020202020202000202064B4
:1070B800697361726D6564202000206E6F207465AD
:1070C8006C20636F6D2000206E6F206770732066E0
:1070D80069782000202062617474206C6F7720200A
:1070E8000062617474207761726E696E6700626114
:1070F8007474637269746963616C0020626174748A
:10710800206572726F7220006C696E6B20717561F8
:107118006C697479006D6167207761726E696E675A
:10712800006D616720637269746963616C00206D2A
:10713800616720206572726F72200025730020003D
:10714800B3060000E803E803E803E8039DFF0164D1
:1071580001000000007B056D3379047C047F048204
:1071680004022A00070E091C1B1215383F36312469
:10717800232A2D70777E796C6B6265484F4641549F
:10718800535A5DE0E7EEE9FCFBF2F5D8DFD6D1C44F
:10719800C3CACD90979E998C8B8285A8AFA6A1B4BF
:1071A800B3BABDC7C0C9CEDBDCD5D2FFF8F1F6E370
:1071B800E4EDEAB7B0B9BEABACA5A28F88818693DF
:1071C800949D9A2720292E3B3C35321F181116030F
:1071D800040D0A5750595E4B4C45426F68616673FF
:1071E800747D7A898E878095929B9CB1B6BFB8AD25
:1071F800AAA3A4F9FEF7F0E5E2EBECC1C6CFC8DD1F
:10720800DAD3D4696E676075727B7C51565F584DCE
:107218004A4344191E171005020B0C21262F283D3E
:107228003A33344E49404752555C5B7671787F6AF1
:107238006D64633E39303722252C2B0601080F1A5E
:107248001D1413AEA9A0A7B2B5BCBB9691989F8A8E
:107258008D8483DED9D0D7C2C5CCCBE6E1E8EFFA7E
:10726800FDF4F3C2C0C0C1C0C0C1C0C0C4C0C0C169
:10727800C0C0C1C0C0C3C0C0C1C0C0C1C0C0C5C0FB
:10728800C0C1C0C0C1C0C000000000182B6D338948
:107298002AB92AE92A062B9F2A272A6D2BDD2B00DB
:00000001FF
